:1000000000000220E57200000D7300000F73000075
:10001000117300001373000015730000000000004E
:100020000000000000000000000000001773000046
:1000300019730000000000001B7300001D73000016
:100040001F730000DD5100008D7700001172000069
:100050001D7200001F7300001F7300001F7300005B
:100060001F7300001F730000993300001F7300000E
:100070001F7300001F7300001F7300001F73000038
:100080001F730000117800001F7300001F73000031
:100090001F7300001F7300001F7300001F73000018
:1000A0001F7300001F7300001F7300001F73000008
:1000B0001F7300001F73000000000000000000001C
:1000C0001F7300001F7300001F7300001F730000E8
:1000D0001F7300001F7300001F730000000000006A
:1000E0000000000000000000000000000000000010
:1000F0000000000000000000000000000000000000
:1001000000000000000000000000000000000000EF
:1001100000000000000000000000000000000000DF
:1004000010B5054C237833B9044B13B10448AFF34E
:1004100000800123237010BD340200200000000082
:10042000E8CB000008B5034B1BB103490348AFF309
:10043000008008BD0000000038020020E8CB00006A
:10044000154B002B08BF134B9D46A3F5803A0021A6
:100450008B460F461348144A121A09F071FC0F4BD1
:10046000002B00D098470E4B002B00D0984700205F
:10047000002104000D000D48002802D00C48AFF305
:10048000008009F015FC2000290007F0D7F909F0D9
:10049000E9FB00BF0000080000000220000000008F
:1004A0000000000034020020F88D01200000000050
:1004B0000000000010F0010310D104280CD90368DB
:1004C000C3F30F1343B1013B9B001A1DC1180979F7
:1004D00011B101339342F9D1184670470023FBE76D
:1004E000037883B11A0601D40130704703F0C003CA
:1004F000C02B08BF0130024610460132037803F0DA
:10050000C003802BF8D0704708B5002103780BB9E1
:10051000084608BDFFF7E4FF0131F7E738B50022D0
:1005200004460D46411C092003F042FA40B1630025
:10053000024643F0010342F8043F0023A34200DBDC
:1005400038BD55F8231042F8041F0133F6E701289F
:1005500038B504DC1C20BDE8384001F023B80D6834
:10056000EA0701D41120F6E74868C30706D4042837
:1005700004D9036803F00F03042B01D00E20EAE72F
:1005800003F07AF86D10002D044603DDFFF7BCFF81
:10059000A84206DA1220DEE72046FFF7A1FF013D60
:1005A0000446012DF8D120787F2808DDDF280ADCF9
:1005B0006378800100F4F86003F03F0318434000C3
:1005C00040F0010038BDEF280ADC637800039B018E
:1005D00080B203F47C630343A07800F03F00EDE7B2
:1005E000F72810DC637880041B0303F47C3300F4E9
:1005F000E0101843E37803F03F030343A078800141
:1006000000F47C60DAE74FF0FF30D8E7486838B58F
:10061000C3070D4606D4042804D9036803F00F026B
:10062000092A04D00B20BDE8384000F0BBBF446865
:10063000C3F30F1364105A1EA2420BD8032194FB7C
:10064000F1F16429A8BF64210329ACBF5918D91C52
:1006500003F0EAF90368C3F30F13013B9C4208D28D
:10066000A31C013464002A6840F8232044F00104EC
:100670004460002038BD01282DE9F84304DC1C202B
:10068000BDE8F84300F08EBF02284E680CD08C689D
:10069000E70709D56410012CB8BF0124F50705D57B
:1006A0004FF0FF30BDE8F8830124F7E7042EF7D9B7
:1006B00033680D6803F00F02042A2DD1E80706D431
:1006C000042D04D92B6803F00F03042B01D00E2056
:1006D000D6E73046FFF7EEFEA042E1DB304602F0FF
:1006E000CBFF0646284602F0C7FF013C0146301901
:1006F00009F0F3FE01460028D2D0012433780BB173
:100700008E4203D3640044F00100CBE73046FFF78C
:10071000E7FE01340646F1E7092A34D177687F10F5
:10072000BC42BDDCE90725D4042D23D92B6803F096
:100730000F03042B1ED1284602F09EFF804604F1D1
:10074000010956F829008542DCD0C2070ED40428DE
:100750000CD9036803F00F03042B07D102F08CFFC0
:100760000146404609F080FE0028CBD0B9454C46F2
:10077000E5DD95E7631C56F82320AA42C2D0BB42B0
:100780001C46F7DD8CE7032A8AD1C3F30F17C3F3A6
:100790004173C3EB8707BC4282DCEB072AD4042DEC
:1007A00028D9286800F00F03032B19D1C0F30F13C9
:1007B000C0F3417005F10408C0EB83003F1A013C0F
:1007C00040440336BC423FF76BAF32194346834285
:1007D000194611D317D10134600040F0010061E7E0
:1007E000042B07D1284602F047FF80462846FFF732
:1007F00061FEE3E70F2043E712F8015F09788D42BD
:1008000003F10103E3D00134DCE708B502F018FF7F
:10081000400040F0010008BDC30711D404280FD9DF
:10082000026802F00F03032B0AD101F00303C3F1A6
:1008300004035B0703F0C04322F0C042134303608C
:10084000704701282DE9F0470546884604DC1C2046
:10085000BDE8F04700F0A6BE4C6814F0010701D1D6
:100860000D20F5E7022802D08B68DA07F8D5D8F812
:100870000060F30700F1A980042E40F2A6803268E0
:100880006410012C02F00F03B8BF0124092B28D1FA
:100890007668022D4FEA660605D0D8F808305B105E
:1008A0009E42A8BF1E46351B0135012225EAE5758B
:1008B000A918092003F07CF8074648B16D000346EB
:1008C00045F00105D8F8002043F8045FA64202DA9B
:1008D0003846BDE8F087013452F8241043F8041F6D
:1008E000F4E7042B43D1304602F0C6FEFFF70CFEBE
:1008F000022D824605D0D8F808305B109842A8BF78
:100900009A46A24504DA0020BDE8F04703F0CAB8D1
:10091000304602F0B1FE0546A74222DB304602F027
:10092000ABFEA94606462846FFF7DAFD0134A2458C
:100930000546F8DAA0EB0905284603F0B3F80746A8
:100940000028C5D002F098FE0446D8F8000002F056
:1009500093FEA9EB060101442A46204609F0CCF992
:10096000B6E72846FFF7BCFD01370546D4E7032B61
:100970002BD1C2F30F13022DC2F34172C2EB8302DB
:1009800005D0D8F808305B109A42A8BF1A46A24298
:1009900006DA002211460320BDE8F04703F008B84C
:1009A000151B0423291D002291FBF3F1032002F003
:1009B000FFFF074600288BD001352946FFF72CFFA3
:1009C000E11C2A4631440430C8E7212040E70028D2
:1009D000F8B504DC1C20BDE8F84000F0E3BD0C686D
:1009E00014F001060FD0641024EAE474E11C002224
:1009F0008910032002F0DCFF054610B12146FFF705
:100A00000BFF2846F8BD042C01D80025F9E725681E
:100A100005F00F05042D19D12046FFF74BFD324696
:100A2000C11C074691FBF5F1032002F0C1FF05460A
:100A30000028E6D03946FFF7EFFE204602F01CFE04
:100A40003A460146281D09F057F9DAE7092DDCD1AD
:100A500067687F100423F91C324691FBF3F10320F1
:100A600002F0A6FF05460028CFD03946FFF7D4FE96
:100A70000434BE42C5DA54F8043FDA0742BFAA196B
:100A8000A3F3480313710136F3E77F2902DC0170F9
:100A900001307047B1F5006F0CDA03468A1162F03D
:100AA0003F0203F8022B01F03F0161F07F0141702A
:100AB00018467047B1F5803F0FDA0B1363F01F0340
:100AC0000370C1F3851301F03F0163F07F0361F010
:100AD0007F014370817003307047B1F5883F0DDAB4
:100AE000F0230370902343708B1101F03F0163F0FA
:100AF0007F0361F07F018370C17004307047000094
:100B00000028F7B50F4603DC1C2000F04BFD0CE07D
:100B10000A6812F001000AD06C4651102046FFF717
:100B2000B4FF011B204602F0C4FF044616E0042A6D
:100B30003BD9136803F00F03092B36D155681C49C4
:100B40006D100124AC420CDD02F0ACFF044628B16C
:100B50003F6802F091FD0126AE421DDD204603B044
:100B6000F0BD013452F8243013F0010601D10D20FC
:100B7000CBE75B107F2B09DDB3F5006F08DBB3F526
:100B8000803F07DB8B42D4BF042600263044D9E7E0
:100B90000226FBE70326F9E7013657F82610CB07B4
:100BA000E5D54910FFF771FFD6E72120ADE700BF7B
:100BB000FF0F010010B5044611F0010011D1042906
:100BC0000ED90B6803F00F03042B09D1084602F07D
:100BD00053FD0146204609F047FCB0FA80F0400979
:100BE00010BD0020FCE700000128F8B50E4604DC2B
:100BF0001C20BDE8F84000F0D5BC4D6815F0010799
:100C000006D1042D04D92B6803F00F02092A01D064
:100C10000B20EEE76C6809681F486410C3F30F13DC
:100C2000A34298BF03F1FF34FFF7C4FF40B1012393
:100C3000BC4201DA0020F8BD013745F82730F7E75C
:100C400031681648FFF7B6FF50B1002CF2D0631C94
:100C50000122013C944045F8232014436C60E9E7ED
:100C60003368DA0701D40D20C3E75B10002B0DDDDC
:100C70009C420BDB05EB830305EB84029A4207D110
:100C80000123013C9C4053601C43E7E71220B0E77E
:100C9000996843F8041FF1E7E7B30000EBB30000E5
:100CA000002310B50B70C3070C4606D50E49421041
:100CB0002046BDE8104009F09BBB28B90B492046EF
:100CC000BDE8104009F0B4BB042801D10849F6E79B
:100CD00009D9036803F00F03042B04D102F0CCFC04
:100CE00004490246E4E710BD20BE0000F0B3000056
:100CF000F6B30000FBB300002DE9F04301288FB0EC
:100D000081460E4607DC1C2000F04CFC05462846B8
:100D10000FB0BDE8F0830B6813F0010440F0A18030
:100D2000042B40F2D5801B6803F00F03092B40D140
:100D3000274656F8273013F0010806D1042B04D9B2
:100D4000186800F00F00092801D02220DCE75B685A
:100D50000137B94504EB6304EBD10122A11802F07D
:100D600027FE054608B90025D1E7640044F00104D8
:100D70004460424600F1080456F822104B680868A7
:100D80005B10C0F30F10984298BF00F1FF3304319D
:100D90000020834207DC013223EAE373BA4204EB0A
:100DA0008304E9DBB3E751F804CF44F820C00130F5
:100DB000EFE7032B40F08C80274656F8270010F011
:100DC0000108C2D10428C0D9036803F00F02032A26
:100DD00038D1C3F30F12C3F34173C3EB82031C4436
:100DE0000137B945E9D10423E11C002291FBF3F15D
:100DF000032002F0DDFD05460028B4D02146FFF7B0
:100E00000BFD00F1040956F82840E10720D4042C1A
:100E10001ED9206800F00F03032B19D1C0F30F1364
:100E2000C0F34170C0EB830003344B46A3EB0902CF
:100E3000824211DB08F101080028A8BF8144B845AF
:100E4000E1DB64E7042A80D1FFF734FB0444C7E701
:100E50002046FFF72FFBE7E714F8012F03F8012BDB
:100E6000E4E700252C4656F82500C20732D40428B2
:100E700030D9036803F00F02042A32D1FFF71AFBBE
:100E800004440135A945EED1204602F00BFE05468B
:100E900000283FF468AF041DB04606EB890958F8F6
:100EA000046BF30728D4042E26D9336803F00F020D
:100EB000042A34D13046FFF7FDFA0746304602F0E7
:100EC000DBFB3A460146204608F016FF3C4421E091
:100ED0002546C8E701A9FFF7E3FE01A809F0CEFA0D
:100EE000CEE7032A7FF431AFC3F30F12C3F341738C
:100EF000C3EB82031C44C4E701A93046FFF7D0FED0
:100F000001A809F0BBFA01A906460246204608F0EE
:100F1000F3FE3444C145C2D100232370F7E6032A0F
:100F2000F8D1C3F30F17C3F34173C3EB87073A46F6
:100F3000311DC8E72DE9F04F002893B00F4607DCBC
:100F40001C2000F02FFB0546284613B0BDE8F08FAB
:100F50000D6815F0010806D1042D04D92B6803F0A3
:100F60000F03092B01D00B20EBE76E687610002EE3
:100F700003DC404602F096FDE5E7012826D04868EC
:100F8000C20723D4042821D9036803F00F03042BDC
:100F90001CD102F071FB0446204609F06FFA0435BB
:100FA000731E8146009303FB00FB05EB860A55F890
:100FB000040FC30771D404286FD9036803F00F022C
:100FC000042A05D1FFF776FA83440AE0384CE3E7B8
:100FD000032A69D1C3F30F12C3F34173C3EB820336
:100FE0009B44AA45E3D1584602F05CFD0546002823
:100FF000AAD0D7F800A0B9F1000F03D0786802F0AA
:101000003BFB0446284602F037FB0AF1040307467F
:101010000193019B53F804AF0193504602F02CFB5F
:101020001AF001030146029302D1BAF1040F04D869
:1010300005A95046FFF734FE05A90846039109F0BB
:101040001DFADDE9023183468BB9BAF1040F0ED9DE
:10105000DAF8000000F00F0CBCF1030F01BFC0F381
:101060000F13C0F341700AF10401C0EB830B384643
:101070005A4608F041FE5F44B9F1000F08D0009BCA
:10108000434505DD38464A46214608F035FE4F44C3
:1010900008F101084645BCD156E705A9FFF700FE57
:1010A00005A809F0EBF98FE702F0E6FAF9E700BFCF
:1010B0008FB80000002810B511DD0B6813F0010493
:1010C00002D05C1024EAE4740122A118092002F085
:1010D0006FFC18B1640044F00104446010BD0024AA
:1010E000F2E70A6838B512F0010436D1042A34D97F
:1010F0001368496803F00F00092818D15068C3F33A
:101100000F134010834298BF03F1FF30151DA0421A
:1011100005DC01330220984205DB002038BD45F88C
:10112000041F0134F3E742F820100130F3E70328ED
:1011300013D1C80704D41320BDE8384000F032BAF8
:101140004910FF29F7D80432C3F30F1302EB8303CE
:101150009A42E2D202F8011BFAE70B2000F022FAD1
:10116000DBE700002DE9F8434E6816F001080F4652
:1011700027D1042E25D9346804F00F03092B10D190
:101180007568C4F30F146D10AC4200D8651E396841
:10119000CB071AD54C10002C01DDA54220DA122015
:1011A00034E0042B04D13046FFF784F90546EEE71E
:1011B000032B08D1C4F30F15C4F34174C4EB8505A8
:1011C000E5E70025E3E74546E1E72F48FFF7F2FCB6
:1011D000B0B109F0A5F890FBF5F404FB1504013457
:1011E000B8F1000F4ED1042E4CD9336803F00F0331
:1011F000092B11D1013456F824402046BDE8F8836C
:1012000039682248FFF7D6FC20B91120BDE8F84321
:1012100000F0C8B92C46E3E7042B2BD1304602F08E
:101220002BFA0546FFF770F9A042B8DB012C1BDC56
:10123000304602F021FA81462846FFF751F9461B55
:10124000304602F02FFC04460028D6D002F014FAF3
:101250008046786802F010FAA5EB09010144324695
:10126000404608F049FDC8E72846FFF739F9013C38
:101270000546DBE7032B05D13444E478640044F0F1
:101280000104BAE70B20C1E7E0B30000EBB30000B4
:101290002DE9F0414C6814F0010688462ED1042C4B
:1012A0002CD923688F6803F00F02092A13D16568CF
:1012B000C3F30F136D10AB4200D85D1ED8F80010B9
:1012C0002848FFF777FC68B3236803F00F03092B66
:1012D0001ED1012317E0032A10D1FA0704D41320EA
:1012E000BDE8F04100F05EB97E10FF2EF7D8C3F3E1
:1012F0000F15C3F34173C3EB8505DFE70B20EFE761
:10130000013344F823709D42FADA0020BDE8F081F1
:10131000032BFAD1033401239D42F6DB04F8016F5D
:101320000133F9E7D8F80010CB0706D5491000299A
:1013300001DD8D4208DA1220D2E70B48FFF73AFCB4
:1013400008B91120CCE72946236803F00F03092BC5
:1013500003D1013144F82170D7E7032B04BF64188F
:10136000E670D2E7E7B30000EBB30000086808B509
:10137000C3071BD4042819D9036803F00F02092AF4
:1013800001D1406808BD032A09D1C3F30F12C3F38A
:101390004170C0EB8200400040F00100F2E7042AF7
:1013A00004D102F069F9FFF7AFF8F4E70B20BDE8CC
:1013B000084000F0F7B80000024A03480B2103F090
:1013C000C9BF00BF88B3000080B300000020704791
:1013D0000420704701207047002002F063BB00200A
:1013E00070470020704700207047002070470020A1
:1013F00070470020704700207047002070470000B1
:10140000024A03480C2103F0A5BF00BF70B40000DE
:10141000D0B400007047000010B510F0010402D0F5
:101420004410204610BD042812D9026802F00F02B1
:10143000042A07D102F020F90A222146BDE8104013
:1014400009F0E0B8032A03D10A2221460430F5E767
:10145000014B0D221A70E4E77402002010F0010223
:1014600010B516D1042802D90268C2F30F1211F088
:10147000010310D1042902D90B68C3F30F1393425F
:1014800016D1043000EB83020331904205D30120D2
:101490000BE00022EBE70023F1E710F8014B11F815
:1014A000013F1CB9B3FA83F0400910BD9C42ECD057
:1014B0000020FAE72DE9F74F804689469A46304FDB
:1014C000304E6AB102233B70012333603368DFF88A
:1014D000D0B00024FC54444504DB03B0BDE8F08FD9
:1014E0003260F3E759F824003168C30707EB0105C0
:1014F000C1F5487105D5244A4310284608F044FF39
:1015000004E0C8B9214A284608F03EFF1C4808F00C
:10151000B5FF3060BAF1000F0CD008F1FF33A342E1
:1015200008DDB0F5487F05D2431C20223A54002242
:10153000FA5433600134CEE7042801D1144AE2E7BB
:101540001BD9026802F00F03042B06D1019102F0AF
:1015500093F8104A01990346CFE7092B03D143685A
:101560005A465B10C9E7032B08D1C2F30F13C2F32D
:101570004172C2EB8303084ABFE70123074ABCE775
:10158000750200209805002020BE0000F0B3000086
:10159000F6B300004BC400004FB700005AB700007C
:1015A00040B70000014B1870002070477402002003
:1015B00010B501F095FD084C231D01461F22184669
:1015C00008F076FF08F05AFF04308008000140F070
:1015D00004002060204610BD500200202DE9F04F8D
:1015E00085B000F1180104690291D0E90232824607
:1015F00001EB8404BD4F4169029800EB8109397801
:1016000003EB820529BB53F82230B94A1E1203F0BE
:101610007F03043552F82330904643F00103184706
:101620009AF8010004F0EAFA00238AF8003021E079
:101630003B7873B92B681E1203F07F03043558F80A
:101640002330EAE7029B221DD31AD82B26DD1A236A
:101650003B70DAF808209AF8023039789AF80100DD
:10166000AA1A921043EA022204F0CEFA00238AF862
:1016700000303B70DAF80830ED1A029BE41AA9EB4F
:101680000309AD10A4104FEAA903CAF80C50CAF818
:101690001040CAF8143005B0BDE8F08F3B782660E2
:1016A0000BB11446D5E72B681E1203F07F031446D6
:1016B00058F823300435B0E7029B221DD31AD82BEB
:1016C00002DD1A233B70C4E72968216039782B1D9D
:1016D00011B114461D46BCE76B681E1203F07F0370
:1016E000144658F82330083597E7029B221DD31A79
:1016F000D82B02DD1A233B70ABE73B7805EB86065F
:1017000026600BB11446A4E72B681E1203F07F037A
:10171000144658F8233004357FE7029B221DD31A64
:10172000D82B02DD1A233B7093E7724B53F8263017
:1017300023603B780BB114468BE72B681E1203F035
:101740007F03144658F82330043566E7694B54F894
:10175000042D43F826203B78002B7FF47AAF2B68CA
:101760001E1203F07F03043558F8233055E7614B10
:10177000009353F82600FFF74FFE834654F8040DFC
:10178000FFF74AFE5844009B400040F0010043F838
:1017900026003B78002B7FF45CAF2B681E1203F011
:1017A0007F03043558F8233037E7029B221DD31AF4
:1017B000D82B02DD1A233B704BE7029B4B4534BF0D
:1017C00059F80C3C012323603B780BB1144640E7E9
:1017D0002B681E1203F07F03144658F8233004359B
:1017E0001BE7029B221DD31AD82B02DD1A233B7064
:1017F0002FE7029B4B450FD259F80C3C06F180466F
:101800005B10C3EB8373033E334459F823302360EA
:101810003B782BB114461CE718233B700023F6E7F6
:101820002B681E1203F07F03144658F8233004354A
:10183000F3E6029B4B4519D259F80C3C54F8042CA2
:101840005B1006F18046C3EB8373033E3344043CD4
:1018500049F823203B78002B7FF4FBAE2B681E1247
:1018600003F07F03043558F82330D6E618233B7085
:10187000F0E7029B4B452DD259F80C3C06F180460F
:101880005B10033EC3EB8373334459F82300FFF727
:10189000C3FD221F834654F8040C0092FFF7BCFDE1
:1018A00059F80C3C009A5B10C3EB837358441E44F8
:1018B000400040F0010049F8260014463B78002B18
:1018C0007FF4C7AE2B681E1203F07F03043558F86F
:1018D0002330A2E618233B70F0E7029B221DD31AA7
:1018E000D82B09DD1A233B70B3E600BF7402002039
:1018F00040B50000C48B012059F8263023603B78A6
:101900000BB11446A5E62B681E1203F07F031446A4
:1019100058F82330043580E654F8043D49F8263061
:101920003B78002B7FF495AE2B681E1203F07F03EB
:10193000043558F8233070E659F826004FEA600B5A
:1019400054F8040DFFF768FD584440003B7840F020
:10195000010049F82600002B7FF47BAE2B681E1295
:1019600003F07F03043558F8233056E6029BA4EBBE
:101970008604A3420BD83B78002B7FF46AAE2B6819
:101980001E1203F07F03043558F8233045E6C5489E
:1019900001F062FE3B78002B7FF45BAE2B681E12D9
:1019A00003F07F03043558F8233036E6002E05EBAC
:1019B0008605FFF65FAE3B78002B7FF44AAE2B68BE
:1019C0001E1203F07F03043558F8233025E654F83F
:1019D000043D042B04D1002E05EB8605FFF64AAE2C
:1019E0003B78002B7FF435AE2B681E1203F07F038B
:1019F000043558F8233010E654F8043D042B04D085
:101A0000002E05EB8605FFF635AE3B78002B7FF404
:101A100020AE2B681E1203F07F03043558F82330E4
:101A2000FBE554F8040CC3070BD54010013800281F
:101A30000ADB400040F0010005EB860544F8040C89
:101A400018E6FFF7E9FCF1E73B78043C002B7FF454
:101A500000AE2B681E1203F07F03043558F82330C4
:101A6000DBE5029B04F10C02D31AD82B02DD1A230A
:101A70003B70EEE5730003F4FF7343F00103236052
:101A8000DAF80830EB1A9D109AF8023043EA052381
:101A90005B0043F001036360029BA9EB03035B104F
:101AA00043F00103A3603412E6B27F4B8AF8024090
:101AB00091463A7853F83630CAF808301AB103F133
:101AC00008054C46C5E503F10C059B681E1203F0A2
:101AD0007F034C4658F823309FE5029B54F8046C72
:101AE0004B452FD1F10720D4042E17D9336803F0CA
:101AF0000F03042B13D1304601F0BEFD08F0BEFCED
:101B0000B0F5487F28BF4FF448700630643003F0CA
:101B10005DFC70B9043DDDF80890ABE507D0002E00
:101B200014BF4FF400700720F0E70A20EEE707200B
:101B3000ECE731469AF8010004F07DF800238AF8BA
:101B40000030E8E759F80C3C57495A106FF003038E
:101B500053430C3B09EB030449F8036059F8083C74
:101B60005A108AF80220D2B2C3F3552351F832201A
:101B7000CAF8082059F8041C4FEA6109029901EBE0
:101B800089093978043402EB830500297FF461ADBB
:101B900052F823301E1203F07F03043558F8233027
:101BA0003BE554F8040CFFF737FC1E288346A4EBF2
:101BB000860425DC00280BDC3B78002B7FF449AD44
:101BC0002B681E1203F07F03043558F8233024E5F8
:101BD00001F076FAABF1030B344E834401F070FA56
:101BE000A0EB0B00B042F9D83B78002B7FF431AD6D
:101BF0002B681E1203F07F03043558F823300CE5E0
:101C000001238AF8003001F05BFA0A385844CAF818
:101C100004002FE554F8040CFFF7FEFBA4EB860448
:101C2000061E0BDC3B78002B7FF413AD2B681E12D5
:101C300003F07F03043558F82330EEE41C4B9E423A
:101C400002DD1D233B7004E501238AF8003001F01A
:101C500037FA4FF47A7303FB06000A38D7E70023FC
:101C60003046A4EB8604134E1A462146FFF722FCA9
:101C70003168114801F01DFF104B316818600E48A3
:101C800003F080FE31680C4803F0DAFF3B78002B4C
:101C90007FF4DFAC2B681E1203F07F03043558F885
:101CA0002330BAE46CB70000CC8301203F420F0020
:101CB00080EE360098050020750200200800002004
:101CC0003B78A4EB8604002B7FF4C3AC2B681E1278
:101CD00003F07F03043558F823309EE4504603F0A8
:101CE000D9FB3B78002B7FF4B4AC2B681E1203F0B9
:101CF0007F03043558F823308FE454F8043CB3BB19
:101D000054F80C3CDA0726D55B105A0042F0010269
:101D100044F8082C002B3BDD5A0042F0010244F845
:101D2000042C54F8082CC3EB620354F80C2CD10794
:101D300020D501335B0043F0010349F826303B789E
:101D4000002B7FF486AC2B681E1203F07F03043552
:101D500058F8233061E4042B06D91A6802F00F0208
:101D6000092A01D15B68CFE719233B7071E45B104E
:101D7000013BCFE7042A08D9116801F00F010929B6
:101D800003D1023352F82330D7E719233B7060E4C4
:101D90000435D4E7029A04EB86039B1AD82B10DC97
:101DA0000122002E06F1FF330EDC3B78002B7FF47E
:101DB00050AC2B681E1203F07F03043558F8233013
:101DC0002BE41A233B7044E422601E460434E8E707
:101DD000029A231D9B1AD82B02DD1A233B7038E48C
:101DE000029B4B452AD254F8040CFFF715FB002840
:101DF00021DD59F80C3C5B1083421CDBC3EB837381
:101E0000184400F180400438A4EB860359F82020E0
:101E10001A606FF0030303FB06443B780434002B85
:101E20007FF417AC2B681E1203F07F03043558F8BB
:101E30002330FFF7F2BB20233B70EAE71823FBE7D0
:101E4000C04B1A68A4EB86031A606FF0030303FB10
:101E500006443B780434002B7FF4FBAB2B681E1246
:101E600003F07F03043558F82330FFF7D6BB54F84E
:101E7000043C042B3B780CBF05EB8605043C002B8F
:101E80007FF4E7AB2B681E1203F07F03043558F88C
:101E90002330FFF7C2BB54F8043C042B1CBF0023C3
:101EA00044F8043C3B78A4F104021CBF05EB860512
:101EB000224613B11446FFF7CCBB2B681E1203F069
:101EC0007F03144658F823300435FFF7A6BB002ED5
:101ED000A4EB860115DC1C233B7000226FF003038A
:101EE00003FB06443B780A600434002B7FF4B1AB5B
:101EF0002B681E1203F07F03043558F82330FFF7D8
:101F00008CBB0B684FF0000C5B1051F82C0010F0EC
:101F1000010202D10D233B70E0E7401083420CF137
:101F2000010CA8BF03466645EFDC5B0043F00102ED
:101F3000D4E7002EA4EB860115DC1C233B700022A5
:101F40006FF0030303FB06443B780A600434002B64
:101F50007FF47FAB2B681E1203F07F03043558F823
:101F60002330FFF75ABB0B684FF0000C5B1051F8A1
:101F70002C0010F0010202D10D233B70E0E740106D
:101F800083420CF1010CB8BF03466645EFDC5B00F1
:101F900043F00102D4E754F8080CFFF73DFA8346FA
:101FA00054F8040CFFF738FAA4EB86038345B4BF5A
:101FB0000420002018606FF0030303FB06443B7805
:101FC0000434002B7FF445AB2B681E1203F07F0313
:101FD000043558F82330FFF720BB54F8080CFFF7FE
:101FE0001BFA834654F8040CFFF716FAA4EB860399
:101FF0008345D4BF0420002018606FF0030303FB67
:1020000006443B780434002B7FF423AB2B681E126C
:1020100003F07F03043558F82330FFF7FEBA54E984
:1020200002014FEA860B8142A4EB0B0B14D104236F
:10203000CBF800306FF0030303FB06443B78043415
:10204000002B7FF406AB2B681E1203F07F030435D0
:1020500058F82330FFF7E1BA042801D80023E7E756
:10206000C307FBD4036803F00F03042BF6D1CB079F
:10207000F4D40429F2D90B6803F00F03042BEDD13B
:10208000FFF7ECF900280CBF00230423D0E754E944
:1020900002014FEA860B8142A4EB0B0B14D1002303
:1020A000CBF800306FF0030303FB06443B780434A5
:1020B000002B7FF4CEAA2B681E1203F07F03043599
:1020C00058F82330FFF7A9BA042801D80423E7E71A
:1020D000C307FBD4036803F00F03042BF6D1CB072F
:1020E000F4D40429F2D90B6803F00F03042BEDD1CB
:1020F000FFF7B4F900280CBF04230023D0E754F8FD
:10210000080CFFF789F9834654F8040CFFF784F9AB
:10211000A4EB86038345ACBF0420002018606FF059
:10212000030303FB06443B780434002B7FF491AA9D
:102130002B681E1203F07F03043558F82330FFF795
:102140006CBA00BF0800002054F8080CFFF764F9CF
:10215000834654F8040CFFF75FF9A4EB860383452C
:10216000CCBF0420002018606FF0030303FB06447B
:102170003B780434002B7FF46CAA2B681E1203F00A
:102180007F03043558F82330FFF747BA54F8043C6E
:10219000042BA4EB860314BF042200221A606FF004
:1021A000030303FB06443B780434002B7FF451AA5D
:1021B0002B681E1203F07F03043558F82330FFF715
:1021C0002CBA54F8080CFFF727F9834654F8040C8E
:1021D000FFF722F95844A4EB8603400040F00100C9
:1021E00018606FF0030303FB06443B780434002BB4
:1021F0007FF42FAA2B681E1203F07F03043558F8D2
:102200002330FFF70ABA54F8080CFFF705F98346A4
:1022100054F8040CFFF700F9ABEB0000A4EB8603C5
:10222000400040F0010018606FF0030303FB064418
:102230003B780434002B7FF40CAA2B681E1203F0A9
:102240007F03043558F82330FFF7E7B954F8080C3A
:10225000FFF7E2F8834654F8040CFFF7DDF800FBC3
:102260000BF0A4EB8603400040F0010018606FF013
:10227000030303FB06443B780434002B7FF4E9A9F5
:102280002B681E1203F07F03043558F82330FFF744
:10229000C4B954F8040CFFF7BFF88346B8B91F233C
:1022A0003B70A4EB8603C3F800B06FF0030303FB9D
:1022B00006443B780434002B7FF4CBA92B681E1214
:1022C00003F07F03043558F82330FFF7A6B954F81C
:1022D000080CFFF7A1F890FBFBFB4FEA4B0B4BF010
:1022E000010BDEE754F8040CFFF796F88346B8B903
:1022F0001F233B70A4EB8603C3F800B06FF0030309
:1023000003FB06443B780434002B7FF4A2A92B681E
:102310001E1203F07F03043558F82330FFF77DB910
:1023200054F8080CFFF778F890FBFBF303FB1B0B4A
:102330004FEA4B0B4BF0010BDCE754F8040CFFF7B2
:102340006BF80028B8BF4042A4EB8603400040F081
:10235000010018606FF0030303FB06443B7804346C
:10236000002B7FF476A92B681E1203F07F0304353F
:1023700058F82330FFF751B9A4EB860B012EDBF898
:10238000000028D1FFF748F8324603460393009235
:1023900007F0C6FF039B009A012BB8BF012390FBF7
:1023A000F3F101FB130313445B0043F00103CBF88B
:1023B00000306FF0030303FB06443B780434002B2A
:1023C0007FF447A92B681E1203F07F03043558F8E9
:1023D0002330FFF722B9FFF71FF80090DBF8040065
:1023E000FFF71AF8009A0130831ACFE7A4EB860BA7
:1023F0005946304601F0F2FC6FF0030303FB06443C
:102400003B78CBF800000434002B7FF422A92B6822
:102410001E1203F07F03043558F82330FFF7FDB890
:1024200054F8080CFEF7F8FF834654F8040CFEF746
:10243000F3FF0BEA0000A4EB8603400040F001002C
:1024400018606FF0030303FB06443B780434002B51
:102450007FF4FFA82B681E1203F07F03043558F8A1
:102460002330FFF7DAB854F8080CFEF7D5FF83469F
:1024700054F8040CFEF7D0FF4BEA0000A4EB8603EF
:10248000400040F0010018606FF0030303FB0644B6
:102490003B780434002B7FF4DCA82B681E1203F079
:1024A0007F03043558F82330FFF7B7B854F8080C09
:1024B000FEF7B2FF834654F8040CFEF7ADFF8BEA3B
:1024C0000000A4EB8603400040F0010018606FF0AC
:1024D000030303FB06443B780434002B7FF4B9A8C4
:1024E0002B681E1203F07F03043558F82330FFF7E2
:1024F00094B854F8040CFEF78FFFC043A4EB860396
:10250000400040F0010018606FF0030303FB064435
:102510003B780434002B7FF49CA82B681E1203F038
:102520007F03043558F82330FFF777B854F8080CC8
:10253000FEF772FF834654F8040CFEF76DFF0BFAAA
:1025400000F0A4EB8603400040F0010018606FF03B
:10255000030303FB06443B780434002B7FF479A883
:102560002B681E1203F07F03043558F82330FFF761
:1025700054B854F8080CFEF74FFF834654F8040C87
:10258000FEF74AFF4BFA00F0A4EB8603400040F050
:10259000010018606FF0030303FB06443B7804342A
:1025A000002B7FF456A82B681E1203F07F0304351E
:1025B00058F82330FFF731B854F80C0CFEF72CFF15
:1025C000834654F8080CFEF727FF8BFB002354F8D2
:1025D000040CCDE90023FEF71FFFDDE90023C0F165
:1025E000200CB0F1200103FA0CFC22FA00F040EAC2
:1025F0000C005CBF43FA01F108436FF00303A4EB46
:10260000860E400003FB06443B7840F00100CEF804
:1026100000000434002B7FF41CA82B681E1203F06A
:102620007F03043558F82330FEF7F7BFA4EB860B81
:1026300059463046FEF73EFD6FF0030303FB0644A8
:102640003B78CBF800000434002B7FF402A82B6801
:102650001E1203F07F03043558F82330FEF7DDBF68
:10266000A4EB860421463046FEF73BFD3B78002B69
:102670007EF4EFAF2B681E1203F07F03043558F889
:102680002330FEF7CABFA4EB860B59463046FEF74F
:1026900069FD6FF0030303FB06443B78CBF80000B1
:1026A0000434002B7EF4D5AF2B681E1203F07F0399
:1026B000043558F82330FEF7B0BFA4EB860421465A
:1026C0003046FEF7E5FD3B78002B7EF4C2AF2B6869
:1026D0001E1203F07F03043558F82330FEF79DBF28
:1026E000A4EB860B59463046FEF740FE6FF003031D
:1026F00003FB06443B78CBF800000434002B7EF447
:10270000A8AF2B681E1203F07F03043558F823305E
:10271000FEF783BF54F8040C00F0AEFF54F8083CF9
:10272000DA072AD4042B0CD91B6803F00F03013BF2
:10273000082B10D8DFE803F0052127230F0F0F0F18
:102740002500C74907F090FEA4EB8603002814BFBC
:10275000002204221A606FF0030303FB06443B7857
:102760000434002B7EF475AF2B681E1203F07F0338
:10277000043558F82330FEF750BFBA49E2E7BA49AA
:10278000E0E7BA49DEE7BA49DCE7029B04F1040B53
:10279000ABEB0303D82B03DD1A233B70FEF759BFC5
:1027A00000F096FC3B78400040F00100206013B13F
:1027B0005C46FEF74EBF2B681E1203F07F035C469B
:1027C00058F823300435FEF728BF029B04F1040BB0
:1027D000ABEB0303D82B03DD1A233B70FEF739BFA5
:1027E00000F06EFCA34B03EA40003B7840F0010090
:1027F000206013B15C46FEF72CBF2B681E1203F05D
:102800007F035C4658F823300435FEF706BF029B71
:1028100004F1040BABEB0303D82B03DD1A233B704D
:10282000FEF717BF00F054FC934B1B6898423DBF66
:10283000C3F5830303F63713C018C01A40003B7872
:1028400040F00100206013B15C46FEF702BF2B6828
:102850001E1203F07F035C4658F823300435FEF760
:10286000DCBE00F035FC844B18603B78A4EB86049A
:10287000002B7EF4EEAE2B681E1203F07F030435AE
:1028800058F82330FEF7C9BE3046A4EB8607012373
:102890007A4E1A463946FEF70DFE3068643002F073
:1028A00095FD10B9043DFEF7E5BE9AF801203168A8
:1028B000734803F0D4F901238AF8003000F000FCDB
:1028C000704A33681268063302FB0300CAF804003A
:1028D0003C46FEF7CFBE3046A4EB8607674E012389
:1028E00000223946FEF7E6FD3068643002F06EFDE6
:1028F0000028D7D0624802F031FFDCE7FEF758FE2F
:102900006FF00303A4EB860B03FB06443B78CBF884
:1029100000000434002B7EF49CAE2B681E1203F0E2
:102920007F03043558F82330FEF777BE3B78A4EBDD
:102930008604002B7EF48DAE2B681E1203F07F03FD
:10294000043558F82330FEF768BEA4EB860B5846D2
:1029500000F0F1FB6FF0030303FB06443B78CBF878
:1029600000000434002B7EF474AE2B681E1203F0BA
:102970007F03043558F82330FEF74FBEA4EB860BD7
:10298000584600F0DAFB6FF0030303FB06443B7884
:10299000CBF800000434002B7EF45BAE2B681E12D3
:1029A00003F07F03043558F82330FEF736BEA4EB5E
:1029B000860B5946304600F0C3FB6FF0030303FB60
:1029C00006443B78CBF800000434002B7EF441AE83
:1029D0002B681E1203F07F03043558F82330FEF7EE
:1029E0001CBEA4EB8604204600F0DCFB3B78002BE9
:1029F0007EF42FAE2B681E1203F07F03043558F8C7
:102A00002330FEF70ABEA4EB860B5946304600F091
:102A100003FC6FF0030303FB06443B78CBF8000094
:102A20000434002B7EF415AE2B681E1203F07F03D6
:102A3000043558F82330FEF7F0BDA4EB8604204699
:102A400000F09CFC3B78002B7EF403AE2B681E123A
:102A500003F07F03043558F82330FEF7DEBD00BFD6
:102A60007CB7000084B700008BB7000092B700006D
:102A700097B70000FEFFFF7FA0050020980500200B
:102A800075020020040000200121304600F044FCC3
:102A90003B78002B7EF4DDAD2B681E1203F07F0324
:102AA000043558F82330FEF7B8BD0021304600F059
:102AB00033FC3B78002B7EF4CCAD2B681E1203F068
:102AC0007F03043558F82330FEF7A7BDA4EB860B2F
:102AD000584600F0E3FB6FF0030303FB06443B782A
:102AE000CBF800000434002B7EF4B3AD2B681E122B
:102AF00003F07F03043558F82330FEF78EBDA4EBB6
:102B0000860B584600F0DEFB6FF0030303FB064420
:102B10003B78CBF800000434002B7EF49AAD2B6890
:102B20001E1203F07F03043558F82330FEF775BDFD
:102B3000A4EB8604204600F099FB3B78002B7EF442
:102B400088AD2B681E1203F07F03043558F823303C
:102B5000FEF763BDA4EB8604204603F03DFC3B7802
:102B6000002B7EF476AD2B681E1203F07F03043534
:102B700058F82330FEF751BDA4EB860B584603F0FE
:102B8000C1FC6FF0030303FB06443B78CBF8000065
:102B90000434002B7EF45DAD2B681E1203F07F031E
:102BA000043558F82330FEF738BDA4EB86042046E0
:102BB00003F088FB3B78002B7EF44BAD2B681E1294
:102BC00003F07F03043558F82330FEF726BDA4EB4D
:102BD000860B584603F08EFB6FF0030303FB06449D
:102BE0003B78CBF800000434002B7EF432AD2B6828
:102BF0001E1203F07F03043558F82330FEF70DBD95
:102C0000A4EB86042146304601F07AFB3B78002B8A
:102C10007EF41FAD2B681E1203F07F03043558F8B5
:102C20002330FEF7FABCA4EB86042146304601F0BF
:102C30008DF93B78002B7EF40CAD2B681E1203F04F
:102C40007F03043558F82330FEF7E7BCA4EB860475
:102C50002146304601F08AFA3B78002B7EF4F9AC2D
:102C60002B681E1203F07F03043558F82330FEF75B
:102C7000D4BCA4EB86042146304601F09DFA3B7893
:102C8000002B7EF4E6AC2B681E1203F07F030435A4
:102C900058F82330FEF7C1BCA4EB860B59463046EA
:102CA00003F00AFD6FF0030303FB06443B78CBF807
:102CB00000000434002B7EF4CCAC2B681E1203F011
:102CC0007F03043558F82330FEF7A7BCA4EB860B2E
:102CD0005946304603F0F8FC6FF0030303FB06444B
:102CE0003B78CBF800000434002B7EF4B2AC2B68A8
:102CF0001E1203F07F03043558F82330FEF78DBC15
:102D0000A4EB860B5946304603F0E6FC6FF0030354
:102D100003FB06443B78CBF800000434002B7EF420
:102D200098AC2B681E1203F07F03043558F823304B
:102D3000FEF773BCA4EB860B5946304603F012FA3B
:102D40006FF0030303FB06443B78CBF80000043428
:102D5000002B7EF47EAC2B681E1203F07F0304353B
:102D600058F82330FEF759BCA4EB860421463046C0
:102D700001F016F93B78002B7EF46BAC2B681E1229
:102D800003F07F03043558F82330FEF746BCA4EB6C
:102D900086042146304601F037FA3B78002B7EF45A
:102DA00058AC2B681E1203F07F03043558F823300B
:102DB000FEF733BCA4EB860B5946304601F09EF972
:102DC0006FF0030303FB06443B78CBF800000434A8
:102DD000002B7EF43EAC2B681E1203F07F030435FB
:102DE00058F82330FEF719BCA4EB86042146304680
:102DF00001F048F93B78002B7EF42BAC2B681E12B7
:102E000003F07F03043558F82330FEF706BC029B1D
:102E1000E31A9B10A4EB8604CAF810302146304612
:102E200002F0DCFC3B78002B7EF413AC2B681E1206
:102E300003F07F03043558F82330FEF7EEBB029B06
:102E4000E31A9B10A4EB860BCAF8103059463046A3
:102E500002F0C4FC6FF0030303FB06443B78CBF89D
:102E600000000434002B7EF4F4AB2B681E1203F038
:102E70007F03043558F82330FEF7CFBB2DE9F84F18
:102E8000224D0023002B03F1FF3706DA01F0DAFAB6
:102E900002F0CEFD02F042FF19270026DFF878800D
:102EA0003046D8F80020B24215DD2B68184C0133AB
:102EB0009342A8BF00232B60D5F80090F02303FBBA
:102EC00009F304EB030AE35CA346EBB1022B04D144
:102ED0005046FEF783FB3B46D4E7012B0ED108B9E1
:102EE00000F0EEF8F02303FB09F39B440949DBF8FB
:102EF0000420821A8A429CBF0222E254F02303FB80
:102F000009F3E35C022BE3D00136CAE7000000209E
:102F10006C7A01203F420F009C0500200B4B0122E0
:102F200000211A61C3F80415C3F808150421C3F879
:102F300010154FF44031C3F804131A60044B4FF4DA
:102F400080611960034B1A70704700BF00A00040F9
:102F500000E100E0C705002004207047F8B5D1E982
:102F6000004514F001002DD015F001002AD06410A6
:102F70001C2C3CD81F4F6D1041F288363B5DAE4291
:102F8000A8BF2E46012B05D00121204604F0D2FD1A
:102F900001233B55184B1B780BB9FFF7BFFF002DE2
:102FA0004FF00003154A0EDC154940F2DC50FF25B6
:102FB000D65CB44204BF21F81300D5540133042B6E
:102FC000F6D10420F8BDD15C8C4203D10C4A22F822
:102FD0001360F6E70133042BF5D10023D15CFF2900
:102FE00001D1D454F2E70133042BF7D1E9E70020F3
:102FF000E8E700BFA8050020C70500201C0000204E
:103000000E00002070B5D1E9004514F001001BD07E
:1030100015F0010018D064101D2C28BF1B24164E7B
:10302000335D012B05D00121204604F083FD0123EF
:103030003355124B6D10A5F110029A42104B04D972
:103040004FF0FF321A60042070BD0E4A1C600E4B18
:1030500093FBF5F313800D4A127812B9FFF75EFF68
:10306000F1E70B4A01219164D2F848150B449BB259
:10307000C2F84035E7E700BFA805002090860100B0
:10308000180000200C00002020A10700C705002028
:1030900000A00040002802DC1C20FEF783BA0120BB
:1030A000704704207047002802DC1C20FEF77ABA23
:1030B0000B68DB0701D40D20F8E700207047000003
:1030C000024B01221A64D3F840057047008000408B
:1030D00008B5FFF7F5FF4FF47A73B0FBF3F008BDC6
:1030E00000487047F8B700001D20704770B5054DC7
:1030F0002B5C8B4204460E4602D004F01BFD2E557D
:1031000070BD00BFA805002070B50024084D2646FC
:10311000635D012B08D10021204604F035FD00211C
:10312000204604F007FD665501341D2CF0D170BD1A
:10313000A805002070470F2070473B207047000013
:10314000F8B50B68DA0707460D4604D40D20FEF7E4
:1031500029FA012007E05B10062B05D103F0D8F80F
:10316000400040F00100F8BDF3D80C4A0C4E52F874
:103170002340335D2BB10021204604F0DBFC00230B
:103180003355012F06DD6B68042B03D10221204645
:1031900004F0D0FC204604F0D7FBE1E7DCB70000E8
:1031A000A805002070B50468E20702D54568EB0762
:1031B00004D40D20BDE87040FEF7F4B964101C2C57
:1031C00023D8124E335D012B18D00121204604F084
:1031D000B1FC01231B2C335510D10D4BDA6E0D4B76
:1031E000202AB8BF4FF0A04302F01F0203EB820376
:1031F000D3F8002742F44072C3F80027A5F34A0130
:103200002046BDE8704004F043BC70BDA805002016
:103210004CC700000003005070B50C68E30704D4ED
:103220000D20FEF7BFF9012070BD64101C2C14D8CE
:10323000012814DD4B68042B14BF002502250A4E1B
:10324000335DAB4204D02946204604F073FC35556B
:10325000204604F0B5FC012803D00020E4E7002557
:10326000EDE70420E0E700BFA805002013B50A4AF7
:10327000044692E8030022686B46042A83E80300B0
:1032800019464FF0020003D100F070FF02B010BDEC
:1032900000F092FFFAE700BFA4B7000010B5084C99
:1032A00063792BB10021052004F044FC00236371F5
:1032B000052004F085FC00280CBF0420002010BD70
:1032C000A805002010B5084CE37A2BB100210B2093
:1032D00004F030FC0023E3720B2004F071FC0028A2
:1032E0000CBF0420002010BDA80500200748084995
:1032F000084A012343604B6053600023C0F8003547
:10330000C1F80035C2F80035704700BF00C0014069
:1033100000100240002002401C2870B504460D46F3
:1033200025D8134E335C012B04D0012104F002FC9C
:10333000012333551C2C12D1FFF7D8FF0D4B1A6F08
:103340000D4B202AB8BF4FF0A04302F01F0203EB41
:103350008203D3F8002742F44072C3F80027291CE7
:10336000204618BF0121BDE8704004F00DBC70BDBF
:10337000A80500204CC70000000300500368D907CF
:1033800002D40D20FEF70EB941680A1F5142514187
:103390005810FFF7C1BF0000F8B5314CD4F84031E8
:1033A000B3B10023D4F84055C4F840312D4B186810
:1033B00000280DDB2C4A1178B1FA81F1490911700E
:1033C00004F0E2FB294B1B882B449BB2C4F8403528
:1033D000234AD2F84431002B37D00021244ED2F8B2
:1033E0004445C2F844113378224D0C3433B12B6874
:1033F000032B03D8204AD05C04F0C6FB2B681E4F79
:1034000001335A4202F0030203F0030358BF534250
:103410002B600022042B194618D00133F81810F83D
:10342000010CFF2801D10122F4E702B1296001213A
:1034300004F0AAFB012333702A68104B33F81230D2
:103440002344074A9BB2C2F84435F8BD4FF0FF331E
:103450002B600023337004F58C435033F1E700BF39
:1034600000A0004018000020C60500200C0000202D
:10347000C5050020A40500201C0000200E0000202F
:10348000094B0A4940F2DC521A805A809A80DA804D
:10349000074A00231370074AFF200870487088709D
:1034A000C8701360704700BF0E0000201C00002091
:1034B000C5050020A4050020024B4FF0FF321A6022
:1034C000704700BF18000020024A0348062101F09F
:1034D00041BF00BFACB7000052BF000038B54FF489
:1034E000E1311D4804F00EF81C4B03210122C3F802
:1034F0000815002404211A61C3F810151A60C3F8D6
:1035000004454FF080430221C3F818150A209A6041
:1035100004F014FA124A2346FF21995401331D2B5B
:10352000FBD1104B104D01221A6000200F4A0423DA
:1035300001461468002CFCD02C681160013B44EA61
:103540000020F6D10A4B01221A6004F035F9BDE8DB
:10355000384001F013B800BFEC7901200080004032
:10356000A805002000D0004008D5004000D1004050
:1035700004D00040F8B506460948094F0C4604F04F
:1035800001F88442A8BF04463546AB1B9C4205DDCA
:10359000384603F0FDFF05F8010BF6E72046F8BDBD
:1035A000EC7901200146014803F0B1BFEC7901201C
:1035B000C3070CD4064B1B68834208D8054B1B6815
:1035C000984204D850F8043C002B18BF18467047A6
:1035D000D0050020CC0500200B4908B501220023AE
:1035E00041F823200133642BFAD1084B1A60084BB1
:1035F000084A1846002106F0A3FB074B40F8043F99
:10360000064B186008BD00BFC48B012008000020D5
:10361000D405002070670100A09D0500C8050020AA
:10362000034B044A1A60044B044A1A60FFF7D4BFE4
:10363000D0050020D4050020CC050020446D0120D9
:10364000044B1B681868C0F30F10023820EAE070C2
:10365000704700BFC805002000B59BB00246054971
:1036600001A806F0C5FE01A802F095F802F056FB8D
:10367000FCE700BF7FB80000C30713D4042802D8BA
:1036800012D00B487047036803F00F03042B01D1DD
:1036900004307047092B09D0064A0748032B18BF8E
:1036A0001046704705487047054870470548704701
:1036B000F0B300006AB8000073B8000059B8000009
:1036C000F6B3000063B80000064B074900201A68F3
:1036D00043F8040CC2F30F12023203EB82038B4255
:1036E000F5D37047D8050020446D01202F4B304A98
:1036F0001868304B2DE9F0411C682F4D136803F01A
:103700000F01072928D81368C3F30F13023302EB04
:103710008302AA42F2D32949002251F82200FFF77E
:1037200047FF41F822000132642AF6D1244A10688A
:10373000FFF73EFF1060234A106810B1FFF738FF13
:103740001060214B214C1E680021F0274FF03C08EF
:10375000B14214DBBDE8F081C3F30F1302EB830326
:103760009A42D0D01968CE0707D4884205D28C423D
:1037700003D351F8041C01B11960043BF0E707FBC7
:1037800001F31A191B5D0BB90131E1E71269551EEE
:1037900008FB012204EB82021832002DF4DB52F800
:1037A000040DFFF705FF013D1060F6E7D00500208E
:1037B000D8050020CC050020446D0120C48B0120D9
:1037C00008000020446D01209C0500206C7A012037
:1037D000C307F0B540D4214B1C68A0423CD3204B1A
:1037E0001D68A84238D850F8043CABBB03680246B9
:1037F000C3F30F13012673B9904242F8046C2BD027
:10380000116851F8043C51F82370176041F82320E7
:10381000013B0A46EFE752F82310CF0702EB830C77
:1038200018D48C4216D88D4214D351F8047C8FB929
:103830000F6807F00F0EBEF1070F08D9CCF8007023
:1038400042F8043C0B680A60C3F30F13E1E741F848
:10385000046CD0E7013BCEE7F0BD00BFD0050020EF
:10386000CC0500200D4930B50D4C0B461A6853F8B5
:10387000045CC2F30F12901C65B18B4214BF0A4660
:10388000002243F8042C01EB800103EB8003A342E8
:10389000ECD330BD12011A60F7E700BFD805002055
:1038A000446D0120144B2DE9F041144C1E464FF09D
:1038B00000083268C2F30F1712070FD07D1C9E421A
:1038C0004FEA850505D018462A46314606F01FFA0C
:1038D00003465A1904352B44C2F80080023706EB20
:1038E0008706A642E5D3E41AA410013C044A240149
:1038F0001C601360BDE8F081D8050020446D0120F4
:10390000C80500202DE9F0419AB0FFF7D9FB214D01
:103910000746002455F824000134FFF759FF642CB2
:10392000F8D11D4B1868FFF753FF1C4B186808B1FE
:10393000FFF74EFF1A4DDFF874800026D8F80030EC
:103940009E4218DBFFF78EFFFFF7D0FEFFF7AAFFBE
:10395000FFF7B6FB134B14491B681B68C3F30F1327
:10396000C21B023B01A806F043FD01A801F013FFB2
:103970001AB0BDE8F0812B7813B90136F035DDE7D8
:103980002C69013C002CF8DB05EB84039869FFF7F8
:103990001FFFF6E7C48B012008000020446D0120C2
:1039A0006C7A0120C805002039B800009C05002071
:1039B0002DE9F8431B4C23681B684D1CC3F30F1300
:1039C0009D42064688461746A1460CDBFFF79AFF44
:1039D00023681B68C3F30F139D4204DB0A20BDE874
:1039E000F843FDF7DFBD08F10202D9F800009B1A89
:1039F0001B0140F82230002340F8043C06F00F067B
:103A0000034646EA0816940043F8046B0119083C83
:103A1000C9F800101C44A34201D3BDE8F88343F861
:103A2000047BF8E7C8050020F8B510F0010704464C
:103A30000E462CD1174B1B68834228D8164B1B68A7
:103A4000834224D9154D28600068012200F00F0040
:103A5000FFF7AEFF2C682F600546C0B12146043049
:103A600051F8042BC2F30F12B242A8BF32469200A3
:103A700006F042F9FFF728FE44F8045CFFF736FE33
:103A80002268074B44F8047C134023602C462046F0
:103A9000F8BD00BFD0050020CC050020446D0120FA
:103AA000F0FF0F00011D0022042091FBF0F1FFF751
:103AB0007FBF38B5054608460C46FFF7F3FF50B107
:103AC000C21C2B46591B8C4206DC002CACBF0419CF
:103AD000041C0023237138BD13F8011B02F8011FD9
:103AE000F0E7F0B502289BB00C4604DC1C20FDF783
:103AF00059FD1BB0F0BD0868C20706D4042804D9DC
:103B0000036803F00F03042B01D00E20EFE74B688E
:103B100013F00107F9D1042BF7D91B6803F00F0349
:103B2000042BF2D18B68DB0701D40D20DFE7FFF710
:103B3000A3FD06466068FFF79FFDA5681AAC014625
:103B400004F8647D6D10304602F088FF2946642336
:103B5000224602F0E5FF204606F090FC0146204692
:103B6000FFF7A7FFC5E7000010B50446ADF5806D6F
:103B700010B9FFF797FF0BE002F097FE0138062817
:103B800027D8DFE800F008081017280423000020D9
:103B90000DF5806D10BD204602F001FF011B20468F
:103BA000FFF787FFF4E7204602F0ADFE400040F04B
:103BB0000100EDE769464FF48062204602F0BDFE49
:103BC000684606F05BFC01466846E9E704210348C5
:103BD000E6E70020CDE70420DAE700BFC8B8000020
:103BE000022838B50C4604DC1C20BDE83840FDF73F
:103BF000D9BC0868C10706D4042804D9036803F0B7
:103C00000F03042B01D00E20EFE76368DA07FAD424
:103C1000042BF8D91B6803F00F03042BF3D1A3681E
:103C2000DB0701D40D20E0E7FFF726FD05466068BD
:103C3000FFF722FDA46801466410284602F00EFF3B
:103C4000214602F04AFFBDE83840FFF78DBF01284A
:103C500038B50C4604DC1C20BDE83840FDF7A2BC9A
:103C60000868C10706D4042804D9036803F00F03C9
:103C7000042B01D00E20EFE76368DA07FAD4042B97
:103C8000F8D91B6803F00F03042BF3D1FFF7F4FC02
:103C900005466068FFF7F0FC0146284602F0DEFEAC
:103CA00002F05AFF400040F0010038BD012870B515
:103CB00005460C4604DC1C20BDE87040FDF772BCD4
:103CC0000868C10706D4042804D9036803F00F0369
:103CD000042B01D00E20EFE76368DA07FAD4042B37
:103CE000F8D91B6803F00F03042BF3D1FFF7C4FCD2
:103CF00006466068FFF7C0FC022D014615D0A46897
:103D0000E30712D56410304602F0A8FE054602F023
:103D1000CCFD012812D1002C02DD0135012C07D188
:103D20002846BDE87040FFF71FBF4FF0FF34EAE7B9
:103D3000284602F042FE013C0546EFE70228EFD19B
:103D4000002CEDDD0135012CEAD000221146284679
:103D500002F05DFE02F031FE013C0546F3E7000093
:103D6000086810B510F001041AD0441007EE904A0C
:103D70009FED187AF8EEE77A67EE877A17EE900AE9
:103D800005F01CFC04F026F80022134B05F06EFC35
:103D900003F0D2FF05F01AFF400040F0010010BD13
:103DA000042812D9036803F00F03042B07D1FFF78F
:103DB00063FC0A22214606F025FC0446D6E7032BC5
:103DC00003D10A2221460430F5E70D20FDF7EAFB76
:103DD000CCE700BFD30237390000D040086808B5EF
:103DE000C30706D4042804D9036803F00F03042B87
:103DF00004D00E20BDE80840FDF7D4BBFFF73CFC23
:103E00000378232B08BF01301022002106F0FAFBB3
:103E100000F10053B3F1804F01D31420EAE74000D2
:103E200040F0010008BD0000024A0348062101F0ED
:103E300091BA00BF98B8000090B800000020704709
:103E40001E20FDF7AFBB1E20FDF7ACBB1E20FDF70B
:103E5000A9BB1E20FDF7A6BB1E20FDF7A3BB1E209D
:103E6000FDF7A0BB1E20FDF79DBB1E20FDF79ABBF2
:103E70001E20FDF797BB1E20FDF794BB024A0348A6
:103E80000B2101F067BA00BF04B900005CB9000063
:103E9000034B01221A60034B18689040104370478F
:103EA000646D0120486D01202DE9F041EFF310828F
:103EB000012302F0010883F310881549154C0968A5
:103EC000154D164E01398B4003274FF00E0C4FF065
:103ED0000B0E002B18D02168296018420AD07246B8
:103EE00011000139FDDC2168316039000139FDDC48
:103EF0005B08EEE739000139FDDC2168316062467C
:103F000011000139FDDCF3E788F31088BDE8F0818A
:103F100020000020586D0120080500500C050050BD
:103F200070B5084E084D002456F824000021FFF714
:103F3000DDF855F8240000210134FFF7D7F8052CEF
:103F4000F2D170BDF4B9000040BD000008B5054BCA
:103F500000221A60044B1B680BB102F045FC0020E4
:103F600008BD00BF606D01205078012010B5041E0F
:103F70000ADA0024074B53F8242001239340064A11
:103F80001360064A136010BDFFF7AEF8A042F0DDE3
:103F9000F0E700BF4CC70000586D01201805005025
:103FA0002DE9F843344B1B680C461BB94FF0FF302A
:103FB000FFF7DCFF246814F0010525D0C4F3474364
:103FC000C4F34720C4F3470240F2596540435B43C2
:103FD00090FBF5F193FBF5F0000240EA0140134637
:103FE000534393FBF5F31843244B1B68202B01BF6D
:103FF000234BC4F3456453F8243043EA0020FFF711
:1040000053FF0020BDE8F883042CFAD9236803F09D
:104010000F03092BF5D154F8046FDFF86080DFF847
:104020006090761040F25967B542EADA54F8042FEE
:10403000D3071FD5C2F34743C2F34720C2F347015A
:1040400040435B4390FBF7FC93FBF7F0000240EA30
:104050000C400B464B4393FBF7F31843D8F8003062
:10406000202B02BFC2F3456259F8223043EA0020F8
:10407000FFF71AFF0135D7E7586D01202000002017
:10408000E4BB000008B50B68DA074CBF5B104FF0CB
:10409000FF3301280DDD4A68042A14BF18222022AC
:1040A000054918460A60FFF745F8FFF75FFF002053
:1040B00008BD1822F4E700BF2000002010B510F062
:1040C000010402D04410204610BD042812D9026811
:1040D00002F00F02042A07D1FFF7CEFA0A22214686
:1040E000BDE8104006F08EBA032A03D10A22214609
:1040F0000430F5E70D20FDF755FAE4E7086810F005
:10410000010370B51CD0FFF7D9FF0346203B5E2B9F
:1041100027D8154C03EB83030022012110462344CA
:10412000052A1AD09E5C052410252E4218BF40187F
:10413000013C4FEA41014FEA6505F6D10132EFE754
:104140000428E3D9026802F00F010429DED1C2F38A
:104150000F13002BDAD00379D8E7400040F00100BC
:1041600070BD0120FCE700BF08BA000038B5086840
:104170000D46FFF7A3FF04466868FFF79FFF621E26
:10418000042A014612D8431E042B0FD8084803EB1B
:10419000830313440568012202FA03F32B430360EF
:1041A000044B1B6813B1204602F01FFB002038BDF2
:1041B000606D01205078012038B508680D46FFF782
:1041C0007DFF04466868FFF779FF621E042A0146F6
:1041D00014D8431E042B11D8094803EB830313445E
:1041E000012202FA03F3026822EA0302054B02608D
:1041F0001B681BB10022204602F0F7FA002038BDF0
:10420000606D0120507801202DE9F04F054685B002
:1042100008680C46FFF752FF022D01903CDD6068F4
:10422000FFF74CFF0746A068FFF748FF0446231D31
:10423000DFF8C8A00293661E4FF00108029B9E4261
:1042400006F1010935D006EB8602531E07F1050B76
:104250003D460393AB4522D0042E19D86A1E042A8A
:1042600016D8039B019ADAF800005919224B4FF037
:10427000010C18EA020E0CFA01F11B6811D001437F
:10428000CAF8001023B162464946284602F0ADFA4A
:104290004FEA48080135DDE701242746C7E74E46C7
:1042A000CCE720EA0101CAF80010002BF0D07246DA
:1042B000EAE73D1D042D1BD8012C19D1DFF83C8005
:1042C000DFF834900026D8F8003004FA05F223EA2B
:1042D0000203C8F80030D9F80030013623B10022BB
:1042E0003146781D02F081FA052E05F10505EAD167
:1042F000002005B0BDE8F08F50780120606D0120EE
:10430000086808B5C30703D5FFF7D8FE054B18604A
:10431000054B1B681BB1034B186802F067FA0020BD
:1043200008BD00BF606D0120507801202DE9F341E8
:104330003F4D4FF441732C68ADF804300A238DF8DB
:1043400006305CBBFFF7ECFDDFF8F480264658F83A
:10435000267001213846FEF7C9FE01360021384695
:1043600003F012FC052EF2D100260DF1040816F818
:10437000087001213846FEF7B9FE013601213846A2
:1043800003F002FC032EF2D1FEF79AFE294B1860CF
:1043900001232B60204602B0BDE8F081012C1CD126
:1043A000244C2668FEF78CFE864298BF801BC728E7
:1043B00001D80024EEE700210420FEF797FE00213B
:1043C0000320FEF793FE00210A20FEF78FFEFEF782
:1043D00077FE022320602B60EBE7022C21D1154BE6
:1043E0001C68FEF76DFE844298BF001BB0F57A6F23
:1043F000DFD3042003F0A8FA0446032003F0A4FA54
:1044000006460A2003F0A0FA34442044C0F53F6079
:1044100003230D3090FBF3F0074B1860012003F0ED
:1044200093FA064A00232B6013600124B2E700BF11
:10443000546D01205C6D0120486D0120646D0120E8
:1044400040BD00002DE9F843434E326852B9434B5A
:104450001B683BB9424B1B68002B74D0BDE8F84386
:10446000FFF764BF3F4D2C6884BB3D4B1B68002B9E
:1044700065D13A4A336810681146002865D13A4F31
:104480003A4EDFF8F4800B60002157F82400FEF765
:104490002DFE56F8249001214846FEF727FEB9F17B
:1044A000220F10D858F82920314B1F2AD8BF4FF0BF
:1044B000A04302F01F0203EB8203D3F8002742F46B
:1044C0004072C3F800270134052CDDD12B68264E3D
:1044D000DFF88890254F002BCCBF03F1FF33042376
:1044E000002156F82300FEF701FE2A68214B53F8FD
:1044F0002280002404EB840101EB0803D9F80010AA
:1045000057F82400194101F00101013403F03CFB8C
:10451000052CEFD12B68012156F82300FEF7E6FDAC
:104520002B68002156F8230003F02EFB2B68013383
:1045300093FBF4F404EB84041C1B2C6003E0FFF7F2
:10454000F5FE002895D1BDE8F883002B97D11360C4
:10455000BDE8F843FFF7E4BC606D0120506D012019
:10456000646D01204C6D0120F4B9000040BD0000D5
:1045700000030050E4BC00004CC700004FF0FF30C7
:10458000FFF7F4BC024A0348092100F0E3BE00BF74
:10459000F8BC000054BD00004FF0805310B51A69FC
:1045A000094B0224C3F8044522F00302884203D3D6
:1045B0000022C3F8042510BDD3F80044002CFBD022
:1045C000C3F808051044F1E700E00140002815BFDA
:1045D0004FF4D2214FF4B4214FF4B4204FF496207D
:1045E000FFF7DABF00280CBF4FF496234FF4B42333
:1045F0001868030E532B0CBF20F07F40002070473B
:10460000064B0122C3F80425D3F80024002AFBD06E
:1046100000220160C3F80425704700BF00E001409C
:10462000002821F07F4141F0A6410CBF4FF49620B5
:104630004FF4B420FFF7E4BF0A4B30B50124C3F8B0
:104640000445002903DC0022C3F8042530BD52F8DC
:10465000044BD3F80054002DFBD040F8044B013933
:10466000EFE700BF00E0014038B54C680234054672
:104670000A462146FFF7E0FF05EB840038BD000045
:10468000124B1B68002B0BBF4FF4B4224FF4D22205
:104690004FF496234FF4B42328B91A1DDB79522B1B
:1046A00008BF1046704782420DD9C378522B0AD1F9
:1046B0004368023300EB8300824204D9C378522B53
:1046C00018BF002070470020704700BF686E0120AF
:1046D0002DE9F0410020B4B0FFF7D2FF0024DFF84D
:1046E000A4800546274626464DBB224D2868FFF785
:1046F00079FF3B463246CDE900401F4902A805F04C
:1047000077FE02A801F047F81C4B1A682B68002BB3
:104710000CBF4FF496234FF4B423D21A4FF47041D8
:1047200064235343009193FBF1F302A8144905F06D
:104730005FFE02A801F02FF834B0BDE8F08169688F
:104740002A6801918B1C1F44D1B2C2F307239C42FB
:10475000C2F30742009102A84146B8BF1C4605F0CB
:1047600047FE02A801F017F82846FFF789FF013637
:104770000546B9E7686E01205EBE00006C6E012040
:1047800008BE00004ABE000070B50020FFF72AFFF7
:1047900005460120FFF726FF0C4B1E68B6FA86F48B
:1047A00085424FEA5414B8BF054620461C60FFF707
:1047B0000DFF074A074B002E18BF1346064A691C17
:1047C0002046BDE870401360FFF72ABF686E0120E5
:1047D00004B0040004A005006C6E012070B5002038
:1047E000FFF700FF02460120FFF7FCFE1F4E204CA2
:1047F000054672B968B94FF4D2214FF49620FFF7FD
:10480000CBFE01212846FFF70BFF1A4B35602360D2
:1048100029E0AA4208DD00233360164B23604FF4E1
:10482000B4212368002017E001233360124B23607A
:104830004FF4D221F5E7120E522A08D000B12360BE
:104840000E4800F0A8FFBDE87040FFF79DBF5A6812
:10485000023203EB820301208B4205D21A68551CF9
:10486000E9D10028D3D170BD2160FCE7686E01203A
:104870006C6E012004B0040004A0050023BE0000FB
:1048800010B50020FFF7FCFE014608B9084610BD30
:104890008478FFF7F5FEDA2C08BF0146F5E7000043
:1048A0002DE9F04F4FF480729FB0604C6048DFF804
:1048B00080B1002105F044FA4FF4807200215D4878
:1048C00005F03EFAD4F80090B9FA89F84FEA581882
:1048D0004046FFF77BFE0294574A584C0020B9F13E
:1048E000000F08BF1446FFF7CBFF064626BB48461D
:1048F000FFF778FE411C4046FFF792FE029BB9F19C
:10490000000FC3F800804E4B14BF4FF496224FF4B3
:10491000B4221C60A21A4FF47041642353430091E7
:1049200093FBF1F305A8474905F062FD05A800F0E7
:1049300032FF1FB0BDE8F08F3568C5F30743A3F120
:104940000A02092AC5F3072547D81BF8051091BBB1
:1049500010223D48DFF8F0A005F0F2F937463A683A
:10496000C2F307218D4209D1C2F307410B2927D099
:1049700013292CD00A2901D1CAF800703846FFF754
:104980007FFE07460028EAD12F4F396881B12046C3
:10499000FFF76AFE0123044657F8231029B1204689
:1049A0000393FFF761FE039B04460133042BF3D10D
:1049B00001230BF805303046FFF762FE064695E707
:1049C000D2B2022ADADC0AEB82025760D6E7102262
:1049D0000021504605F0B4F9D0E7A3F11502082AEA
:1049E000E9D8144A525D002AE5D1152B0CBF314697
:1049F000002130460368C3F30742152A0FD01D2A51
:104A000008BF0021FFF73CFE0028F3D119B1204672
:104A1000FFF72AFE0446074A01235355CBE7C3F3A9
:104A200007239D4208BF0146ECE700BF686E0120E6
:104A3000686D0120706E012004A0050004B0040020
:104A40006C6E0120EDBD0000548D0120FFF728BFE2
:104A50002DE9F84FDFF8A8B0274F03339246042220
:104A600093FBF2F6DBF80030B41C002B3B684FEAF6
:104A700084040CBF4FF4B4224FF4D22223449A4250
:104A800081460D46B84614D2FFF70AFFDBF8003026
:104A9000002B3B680CBF4FF4B4224FF4D2222344C6
:104AA0009A4206D2154800F076FE00273846BDE847
:104AB000F88F2D025FFA8AF141F0A441ADB2D8F827
:104AC00000700D434FEA094101F47F012943384644
:104AD000FFF796FD07F108053146381DC8F800506C
:104AE000FFF78EFD1EB10A9A2846FFF7A5FD083C88
:104AF0002544C8F80050D9E76C6E0120C7BD0000FE
:104B0000686E012030B59BB0FFF768FE00214FF4BE
:104B1000FF621D4805F014F9FFF7B2FE1A490024A0
:104B2000A0B9194B024653F8301001B101320130DF
:104B3000FF28F8D1154901A805F05AFC01A800F09A
:104B40002AFE134800F027FE1BB030BD0368C3F3F4
:104B500007420A2A0BD1C3F30722FF2A04D001EB34
:104B6000C20541F832002B71FFF78AFDD8E7132AFE
:104B7000FAD1C3F30723FF2B1EBF01EBC30241F899
:104B800033401471F0E700BFCC83012093BE0000D6
:104B9000A7BE00000A4B0022C3F8002101225A6080
:104BA000D3F80021002AFBD00022C3F80C210122F7
:104BB0009A60044B0222C3F880211A60704700BF3C
:104BC0000010004000E100E0074B0222C3F8802003
:104BD000064B0022C3F8102101221A61D3F81021DC
:104BE000002AFBD0704700BF00E100E00010004049
:104BF00008B504490A780AB1FFF7E6FF00200870FB
:104C000008BD00BF716F01204FF08053586E400007
:104C100040F0010070470000024B1868400040F06F
:104C200001007047F46F0120024B1868400040F00B
:104C30000100704724000020024B1868400040F03B
:104C400001007047F86F012070B504460D46164606
:104C5000FEF73EFA4FF0805301225B6E6270E27005
:104C6000020A23F00043A271020CE2711A0A002129
:104C700060716372000EA2721A0C1B0E2670A17076
:104C800025712072E272237370BD000010B5054CCF
:104C9000204605F0F3FB01462046BDE81040FEF734
:104CA00008BF00BFFD6F0120104B1B685A1C10B5D8
:104CB00014D0CBB1012B13D0022B13D0042B13D063
:104CC0000B4C0C4A052B08BF1446204605F0D6FBBA
:104CD00001462046BDE81040FEF7EBBE064CF4E767
:104CE000044CF2E7054CF0E7054CEEE72800002005
:104CF0003DBF000043BF000038BF00008BB700007D
:104D000084B7000010B521480278002A3DD14FF049
:104D10008043C3F8002101221A60D3F80021002A41
:104D2000FBD01B4B1B4C00220721C3F80C25C3F8FA
:104D300008151949C3F81025C3F81C15C3F8242514
:104D40000121C3F82C250822C3F83015C3F8142517
:104D5000C3F818450224C3F834454FF6FF74C3F86E
:104D60003C450E4CC3F838451824C3F85445C3F8E5
:104D70000423D3F8002242F01002C3F80022084AAC
:104D8000C3F80425FFF706FF017010BD716F012005
:104D900000100040200004027469627521100100B7
:104DA000726F0120F8B5104B1B7804460BB9FFF762
:104DB000A9FF0E4E3378ABB10D4A1278D21A02F029
:104DC00003010C4A02EB411202F1200710685168FE
:104DD000254603C50832BA422C46F7D1013B337051
:104DE0000120F8BD1846FCE7716F0120FC6F01201F
:104DF000706F0120726F012030B5002889B02ADD64
:104E00000D6815F0010426D1042D26D92B6803F076
:104E10000F03092B21D16B683F2B1EDD6846FFF77E
:104E2000C1FFB0B19DF800200435A242A8BF1DF813
:104E3000043004F10104A6BF5B0043F00103012329
:104E4000202C45F8043FF0D1054BDDF809201A600D
:104E5000042009B030BD0020FBE72046F9E700BF81
:104E6000F86F012030B5384B1B788BB00BB9FFF7CA
:104E700049FF02A8FFF796FF10B900200BB030BD24
:104E80009DF808300B2BF8D99DF80930012BF4D18F
:104E90009DF80B30012BF0D12C4D2D4C2D4ADDF817
:104EA000111000232B6023709DF80C3013602A4AE8
:104EB000116023B9DDF815302B6000230FE0012BC2
:104EC00011D1DDF815309DF819202B600DF11A0174
:104ED0000E239342A8BF134600229A4230D10022EB
:104EE000E2540420CAE7022B05D19DF815201223B5
:104EF0000DF11601EDE7042B0DD10AAA6B4652F80D
:104F0000130D516803C3DDE9000102F089FE04F0CE
:104F10005DFE2860D1E7052BCFD10AAA6B4652F877
:104F2000130D516803C3DDE9000102F079FE04F0BE
:104F30004DFE9DF81D2028600A230DF11E01C8E7D3
:104F4000885CA0540132C8E7716F0120F46F012022
:104F5000FD6F012028000020F86F012010B5154BCF
:104F60001B7804460BB9FFF7CDFEFFF72DFE124B61
:104F70000022C3F80445C3F8002101221A60D3F8C7
:104F80000021002AFBD00022C3F80C2101229A60E4
:104F9000094AD2F80C31002BFBD0084B1978084B8A
:104FA00003EB4113C2F80435FFF70EFEBDE81040D5
:104FB000FFF7F0BD716F012000100040706F0120FD
:104FC000726F012000B5002889B01DDD0B6813F059
:104FD000010219D1042B17D9196801F00F01092911
:104FE00012D159683F290FDD043353F8040F10F034
:104FF000010118BFC0F347010DF802100132202A49
:10500000F3D16846FFF7AAFF002009B05DF804FB62
:10501000002810B511DD0C68E3070ED56410532C81
:105020000BD8074B1B780BB9FFF76CFEFFF7CCFDD5
:10503000044BC3F80845FFF7ADFD002010BD00BFCD
:10504000716F012000100040002810B50DDD0C68C4
:10505000E3070AD56410FF2C07D8054B1B780BB962
:10506000FFF750FE034BC3F82445002010BD00BFDE
:10507000716F012000100040002813B515DD0C6889
:10508000E10712D564100A4A0A4B072CCDE9002328
:105090000BD8094B1B780BB9FFF734FE02AB1C444D
:1050A000064B14F9082CC3F80C25002002B010BDE3
:1050B000E2ECF0F4F8FC0004716F012000100040F5
:1050C00070B5002888B020DD086810F001041CD1FC
:1050D00004281AD9036803F00F03042B15D1FEF737
:1050E000CBFA064605F0CAF9122828BF1220054659
:1050F00000F10D0202216846FFF7A6FD8DF80D5064
:10510000A54205DC6846FFF729FF002008B070BD06
:105110000DEB0403325D9A730134F1E72DE9F041A0
:10512000012888B00D4630DD086810F001042CD14C
:1051300004282AD9036803F00F03042B25D14B68F8
:10514000DB0722D5FEF798FA804605F097F96D68DF
:105150000E2828BF0E206E10074600F11102012113
:105160006846FFF771FD6B128DF80D606D14360EF9
:105170008DF80E308DF80F508DF810608DF811708D
:10518000A74206DC6846FFF7E9FE002008B0BDE84C
:10519000F0810DEB040318F804209A740134EFE752
:1051A00030B5002889B016DD0C68E30713D565100B
:1051B000684610220021FFF747FD63128DF80D505D
:1051C00064142D0E68468DF80E308DF80F408DF862
:1051D0001050FFF7C3FE002009B030BD174BD3F8C5
:1051E000002122B10022C3F8002101229A60D3F8E5
:1051F0000C2102B30021C3F80C11D3F80024012ABA
:105200000F4A19D1D3F848355B4213600D4A137821
:10521000032B9CBF013313700B4A1378013303F047
:1052200003031370094A02EB4313044AC2F804351E
:10523000024B01229A6070471160F9E700100040AC
:1052400024000020FC6F0120706F0120726F01208C
:10525000024A0348102100F07DB800BFB8BE00002C
:10526000AFBE0000044A05491368C8540133C3F3B4
:1052700009031360704700BF2C7401202C700120BB
:1052800070B51149114A0B68834202DC00230B60A0
:1052900017E0855CA5F1FA06012E00F1010405D89E
:1052A0009C420FDAA55C013D1F2D01D92046EBE79A
:1052B0000446151A165D2E550134A342FADC181A5D
:1052C000086070BD1570FAE7387801203874012045
:1052D00008B5FDF7F5FE074B1A68824284BF00222D
:1052E0001A601B68C01A44F62063984294BF0020DD
:1052F000012008BD2870012070B5094C094D0A4EE7
:1053000023682A68934200D170BDF05CFEF74AF929
:105310000028F9D023680133C3F309032360EFE7C2
:10532000307401202C7401202C70012070B5074EC0
:10533000074D044633682A689B1ADB43C3F309030D
:10534000A34200DB70BDFFF7D7FFF3E72C74012009
:1053500030740120F0B5074D2B680B2B08DC064F8D
:105360000C245C433E19C6E90112013338512B600D
:10537000F0BD00BF34740120648D012008B5FCF736
:105380001BF8FFF7FFF8FCF73BF8FEF79DF8FEF778
:105390004BFDFEF773FDFFF75BFF01F013F801F023
:1053A00027FABDE8084001F05BBC000008B54FF4E7
:1053B00016620021034804F0C3FC034B00221A606C
:1053C00008BD00BF6C7A01209C050020064B074AEF
:1053D0001B6812689B1ADB43C3F309038342D4BFE3
:1053E00000200120704700BF2C7401203074012080
:1053F000F8B507460E4614461D4673B90320FFF75D
:10540000E5FF10B3FA20FFF72DFFF8B2FFF72AFFF0
:10541000F0B2BDE8F840FFF725BF501DFFF7D6FFFB
:1054200098B1FB20FFF71EFFF8B2FFF71BFFF0B2A9
:10543000FFF718FFE0B2FFF715FFC4F30720FFF7EF
:1054400011FF2E46731B9C4200DCF8BD16F8010BC1
:10545000FFF708FFF6E70000F8B50C4E0C4D0024EE
:10546000F0273368A34203DCBDE8F840FFF79EBF96
:1054700007FB04F359195B5D2BB100231A464978E9
:105480001120FFF7B5FF0134EBE700BF9C050020BA
:105490006C7A0120F8B50E4C0E4E07460025BC4232
:1054A00005F1010511D0237853B100231A46617824
:1054B0001120FFF79DFFF0220021204604F040FC60
:1054C0000A2D04F1F004EAD1F8BD3560F8E700BF19
:1054D0006C7A01209C0500202DE9F04F12F00106A6
:1054E000ADF54F7D82468B4617D001238DF81430E1
:1054F00042FA03F354128DF8153052141B0E8DF836
:1055000017208DF818308DF8164005AB0522FFF7EF
:105510006FFF0DF54F7DBDE8F08F042A2CD911687F
:1055200001F00F03042B38D105AD022310462B7078
:10553000FEF7A2F8044604F0A1FFB0F5487F034649
:1055400004F1FF31A8BF4FF448739E4206F10102F7
:105550000DD1B0F5487F06D96D4B19889B78ADF811
:1055600032138DF834332B4659465046CFE7164652
:1055700011F8012FAA55E8E740F0C680A2F1040C0B
:10558000DCF100024FF0030342EB0C028DF8143003
:105590008DF8152005AB0222E6E7092B40F091803B
:1055A000154604238DF8143055F8043F4FEA63087C
:1055B000B8F1200F8DF815804FEA6323A8BF4FF094
:1055C00020088DF816308DF8178006AC03220521CF
:1055D000B04502DC05ABE21AC6E755F8040F10F03F
:1055E000010706D1042847D9036803F00F03022BF3
:1055F0000DD14FF0010323704310637047121B0E4F
:105600004014A770E070237105340136E0E7042BE5
:1056100030D123464FF0020C03F802CBCDE9012133
:1056200000930393FEF728F8814604F027FF0C2827
:10563000DDE901210AD8009B6070874201D1DC19A5
:10564000E3E719F80740DC550137F6E723460C205D
:1056500003F8010F09F1FF3009F1080910F8017F83
:1056600003F8017F4845F9D12E23E3722373637356
:105670000E34CAE7012B08D12346071F03F8022B7B
:105680007842784160701C46BFE7092B09D104239A
:1056900023704368581060705B12A370E770043485
:1056A000B3E7032B0AD121700368C3F30F10C3F3D0
:1056B0004173C3EB800363701B12EEE72770013464
:1056C000A3E7032B7FF425AF05238DF81430C1F336
:1056D0000F13C1F34171C1EB830164294FEA212308
:1056E0008DF81510A8BF64218DF816308DF81710AD
:1056F00003328E4205AB01DB0A1D35E7334412F855
:10570000010F18710136F4E7002A7FF402AF35E784
:1057100000B400000F4970B5F022002402FB04130E
:105720005D78854203D001340A2CF7D170BDF02298
:105730001846002104F004FB074A1368013BA3420A
:1057400000D11460002329461A461120BDE870409C
:10575000FFF74EBE6C7A01209C05002030B5B3B037
:1057600032AC0223054604F8C83D04F087FEC72882
:1057700028BFC720691E0023984207DC421C23462D
:10578000FE211420FFF734FE33B030BD013311F891
:10579000012FE254F0E770B5B2B032AC02230546F7
:1057A00004F8C83D04F06AFEC72828BFC720064693
:1057B0000023681E9E420BDC06F13200FFF7B6FDA7
:1057C0002346721CFF211420FFF712FE32B070BD79
:1057D000013310F8012FE254ECE700002DE9F04FFF
:1057E0000128B9B08146884603DC1B20FBF7DAFEAE
:1057F00058E00868C2072BD4042829D9036803F0AD
:105800000F03042B24D1FDF737FF0546D8F8040019
:10581000C3071FD404281DD9036803F00F03042B0A
:1058200018D1FDF729FF0646214BDFF890A01B6831
:1058300003930027039BBB420EDC00962B461D4AB8
:10584000C82106A804F0A0FD06A8FFF7A4FFCCE736
:10585000194DDBE7184EE7E70C2303FB07F202EBD9
:105860000A03294652F80A00049304F0FDFD049B44
:10587000044618B9D3E9013B9C4201DB0137D9E763
:105880000BEBC40231465BF834000593049204F03C
:10589000EBFDDDE9042340B9536808F10801A9F1E3
:1058A0000200984739B0BDE8F08F0134E4E700BF4B
:1058B0003474012014C000008FB80000648D0120F2
:1058C0002DE9F0411F4F204AD7F8008005460023FC
:1058D000F02098450EDC0024F02000FB04F1531862
:1058E000565C8EB101340A2CF7D11848BDE8F0415E
:1058F000FFF751BF00FB03F154186478AC4201D1AB
:10590000515CE9B90133E4E7F0223146184604F06E
:1059100017FA0F49457051F8351085700222A045DD
:105920000270C0E90212C0E9046601DC01343C6087
:10593000002329461A461020BDE8F041FFF758BD64
:10594000BDE8F0819C0500206C7A01205DC4000058
:10595000CC83012070B5FFF77FFD094EFF246FF067
:10596000070505FB046393F8FC37043B012B03D8C0
:10597000E043C0B2FFF7A4FF013CF2D170BD00BF0D
:10598000CC8301202DE9F8431D4E07460D46002427
:10599000B046E3009A191279062A01D0032A23D1CE
:1059A00058F80300836803F07F031C2B1CD1C368E5
:1059B00003F07F02042A17D1026902F07F02192A3C
:1059C00012D11B0A00EB83001030FDF755FE03785F
:1059D000814633B104F052FDA84205D100239D4217
:1059E00007DCE0B2FFF76CFF0134FF2CD1D1BDE83A
:1059F000F88319F80310FA5C9142F5D10133EEE710
:105A0000CC830120F8B5094F0546FF246FF0070647
:105A100006FB047393F8FC37AB4203D1E043C0B2FA
:105A2000FFF74EFF013CF3D1F8BD00BFCC8301204E
:105A30002DE9F84FFDF744FB584B1A68824284BFAA
:105A400000221A601A6842F20F71821A8A420BD938
:105A50005349186000235A181279073A022A0FD9BD
:105A60000833B3F5FF6FF6D1BDE8F88F0720FFF7D5
:105A7000C9FF8AF800802EE00820FFF7C3FF3FE04F
:105A8000FDF726FB002814BF044601240020FDF783
:105A900005FC81460020FDF715FC424D424E0746AD
:105AA000B9F1000F17D02B68002B70D133682C6030
:105AB000002B6FD0DFF8F8B0DFF8F0A09BF80030D3
:105AC0004FF00108002BD1D10920FFF79BFF8AF886
:105AD00000808BF80080AFB133689BB92B683460CD
:105AE0001BB3DFF8C8B0DFF8C8A09BF800304FF058
:105AF0000108002BC0D10920FFF784FF8BF800803C
:105B00008AF800802B6883B1284A1178904661B9E1
:105B10009C4238BF2C602B68E31A312B05D9072033
:105B2000FFF770FF012388F80030326882B1204B04
:105B30001978984661B9A24288BF34603368E41A84
:105B4000312C05D90820FFF75DFF012388F80030CC
:105B50002B685BB1B9F1000F08D1144C227812B94F
:105B60000720FFF74FFF00232B6023703368002BC3
:105B70003FF47AAF002F7FF477AF0D4C227812B943
:105B80000820FFF73FFF0023336023706CE7002FEE
:105B9000A2D1B9E7002FA1D1B4E700BF2470012042
:105BA000CC830120147001201C700120187001208A
:105BB0002070012037B50546FFF74EFC02A80024EF
:105BC00040F8044DFDF752FB21462046FEF7BEF992
:105BD000FEF738FCFDF78AFBFDF752FCFDF76CFC85
:105BE000FEF7CCFCFDF790FA25B1FDF7F5FC024875
:105BF000FFF7D1FD03B030BD4EC4000000230146C5
:105C00001A461120FFF7F4BB07B513128DF80120D7
:105C10008DF802301314120E8DF800108DF8033039
:105C20008DF8042001466B4605221320FFF7E0FBA8
:105C300003B05DF804FB0A4601461220FFF74CBC96
:105C400070B50C46054601F13200FFF76FFB2B469D
:105C5000224600211B20BDE87040FFF7C9BB10B4ED
:105C6000144603460A46142021465DF8044BFFF70C
:105C7000BFBB000030B5084C01444FF0FF338842F1
:105C800001D3D84330BD10F8015BDAB26A4054F852
:105C9000222082EA1323F2E730C00000FE2837B545
:105CA000044614D80B4B53F8300080B141680830DB
:105CB0008900FFF7DFFF02AD45F8040D0920FFF76B
:105CC00035FB2B46042221461720FFF791FB03B03A
:105CD00030BD00BFCC830120F8B50746FEF7D0FDEC
:105CE0004FF0FF3504460CB92846F8BD2668C6F3C8
:105CF0000743152B0CD104F10801384604F0B4FB1E
:105D000008B9C6F307252046FEF7BAFC0446EAE7C1
:105D10001D2B08BF4FF0FF35F5E700002DE9F047D8
:105D2000BF4CC04D9CB0FFF7E7FA2068C0F580611A
:105D30002844FDF71FFC23680344064623607BB11B
:105D4000B94F002E0FDC2B78FA2B40F030812368FE
:105D5000022B16DCFFF7BCFA10B10120FFF790FA16
:105D60001CB0BDE8F0872068C0F580612844FDF7CD
:105D700001FC2368034406462360FDF7A1F938605F
:105D8000DFE76878AC78831E182B00F20681DFE825
:105D900013F019002D0031003500380041000401D6
:105DA0004B0080008A008E00A400E000F100040196
:105DB00004010401040104010401040104010401BB
:105DC0000401FF00FF2C0FD02046FFF7A3FC974AE9
:105DD000002342F8343002EBC40221461371132031
:105DE00000931A46FEF734FE0320B7E72046FFF77C
:105DF00067FDF9E72046FFF78DFCF5E7FFF7AAFD01
:105E0000F2E7FFF729FB0020FFF7D4FE8848FFF7F1
:105E1000C2FCE9E7632CE7D8864B214653F82420DF
:105E20001520FFF759FBDFE7FEF72AFD6FF00708A3
:105E30000446002CD8D02768C7F30743152B04D09D
:105E40002046FEF71DFC0446F3E704F10806304641
:105E500004F014FB05460530FFF768FAFB20FFF756
:105E600001FA1D20FFF7FEF9C7F30720FFF7FAF943
:105E7000E8B2FFF7F7F9C5F30720FFF7F3F9A8EB4E
:105E80000407F3199D42DBDD16F8010BFFF7EAF971
:105E9000F7E7002300931A4619461D20FEF7D8FDA8
:105EA000FDF79AFBA0E72046FFF7F8FE9CE7FDF719
:105EB00017F9614A00906421604B03A804F064FA6A
:105EC000022303A88DF80C3004F0D8FA03AB024685
:105ED00000211620FFF78CFA86E7544F002557F86B
:105EE000354007EBC5035CB3D4F8048093F804A0F5
:105EF0004FEA8806B01DFFF719FAFB20FFF7B2F949
:105F0000012006F10109FFF7ADF9E8B2FFF7AAF9A0
:105F10005FFA89F0FFF7A6F9C9F30720FFF7A2F9A6
:105F20005046FFF79FF9083404EB0609A1450BD84A
:105F3000FFF7E2F906EB080001F05CFCFFF7DCF983
:105F40000135FF2DCBD14FE714F8010BFFF78AF98C
:105F5000ECE70024FFF780FA22462146009423460E
:105F6000DA20FEF775FD4FF4FF6221462F4803F05B
:105F7000E7FE95E7012C02D1FEF7AAFB34E7022CDD
:105F800002D1FEF763FD2FE70120FFF713FE2BE799
:105F900000231A4621461A209CE7A0F1C803052BCE
:105FA0003FF622AF00221146FBF734FA1CE7FB2B29
:105FB0007FF4D3AE2268042A7FF7CCAEB5F8037025
:105FC00040F2F6339F423FF7C8AE3B1D9A427FF73F
:105FD000C1AEEB5CFE2B7FF4C0AE6878AC781B28BA
:105FE00007F1FF367AD02DD807285ED0082837D0A1
:105FF00001282CD1FF2C11D02046FFF78BFB6D79A7
:106000000F4B00932146BB1E2A460A20FEF720FDB7
:10601000064B43F8340003EBC4042571781D9DE65C
:10602000387801203874012028700120CC830120A9
:1060300030C40000C48B012047C4000042C40000EB
:106040003E7401201D285BD04DD31E2870D0A0F1D6
:10605000C803052BE2D83F4A3146FBF7DBF9DDE701
:10606000632CDBD86B79022B0CD0032B14D0012BC3
:10607000D4D1D5F80630384A5B0043F0010342F82A
:106080002430CBE7002EC9DDB91E3448FDF711FDE1
:10609000314B43F82400C1E7AB79002B2E4B0CBFEA
:1060A0000022042243F82420B8E7632EB6DC3246EF
:1060B000284903A803F020FE1CAB1E4403A80023BC
:1060C00006F8643CFFF708FE0028A7DB224B2146B8
:1060D00053F820201520FFF7FFF99FE731461D48B0
:1060E000FFF750FC9AE7FF2C98D06A79022A95D8DE
:1060F0001A4B00932146BB1E0B20FEF7A9FC8DE72F
:10610000632EA8BF6326002303A9B3420BDB1CAA9E
:1061100026EAE6731344002203F8642C152000914C
:10612000731C2146E9E7EA185279CA540133ECE7B7
:10613000012C7FF473AF002E7FF770AF6B791BB12A
:10614000322BA8BF32231C4664235C43044B1C60E3
:1061500064E700BF3D740120C48B01203E74012020
:1061600004000020084B01221A60084A1368002B23
:10617000FCD0074B1868042390FBF3F0063840006E
:1061800040F00100704700BF00C0004000C1004067
:1061900008C500400120704710B5064C204600F0AD
:1061A0008BFE0549204600F0EDFE044B01221A60EB
:1061B00010BD00BF74780120801A06003C780120D1
:1061C00010B5064C204600F077FE0549204600F049
:1061D000D9FE044B01221A6010BD00BF30790120A6
:1061E000801A06004078012010B501210D20FCF72F
:1061F0007DFF094C01210E20FCF778FF00210F20C4
:10620000FCF774FF204600F099FD20461021BDE800
:10621000104000F0A9BD00BF547801202DE9F843DB
:106220000C68E30704D40D20BDE8F843FBF7BAB9C6
:1062300064102FD4FCF758FFA0422BDB002120462E
:10624000FCF754FF4FF4FA620121204601F00AFBEB
:1062500000B3DFF86C8000254FF001090027072606
:106260004FF47A720121204601F0FCFA90B12828FF
:10627000C4BF09FA06F31F4316F1FF36F0D205F842
:1062800008700135052DE9D1012206210920FDF70D
:106290008FFB08B900200FE003460B2243F8042FC0
:1062A000064900F1180411F8012F520042F00102D2
:1062B00043F8042F9C42F6D1BDE8F88343780120CF
:1062C0004478012010B50468E30704D40D20BDE82C
:1062D0001040FBF767B96410FF2C01D91720F6E7CF
:1062E000FFF782FFE1B2024800F061FD002010BD1F
:1062F0005478012008B5FFF777FF0021034800F02C
:1063000056FD400040F0010008BD00BF5478012058
:10631000274A82B001210023ADF80630C2F8F015FB
:10632000C2F8001519461A0102F1804202F5E04256
:106330000133082BC2F81415C2F81015F3D11C4B09
:106340004FF4E062C3F818250422C3F81425C3F8FB
:1063500010250DF10602C3F82C260122C3F83026C1
:106360001A60D3F80021002AFBD00022C3F80021D4
:1063700001225A600E4B1A46D3F804110029FBD0B3
:106380000021C3F8041101219960D2F81431002BC7
:10639000FBD00020C2F81401C2F80005BDF8063099
:1063A0001BB28342C8BFA3F50B70400002B0704718
:1063B0000070004008B5FFF7ABFF400040F001005F
:1063C00008BD0000024A03480A21FEF7C3BF00BF10
:1063D00074C40000C4C4000070B50668F10705D598
:1063E0004568EA0702D58468E30704D40D20BDE8B8
:1063F0007040FBF7D7B87610802E01D91520F6E74C
:106400006D10FF2D01D91620F1E76410FF2C01D982
:106410001720ECE70A4B1B680BB9FFF7BDFEF1B282
:10642000084800F02DFEE9B2064800F00DFDE1B28B
:10643000044800F009FD034800F08DFE002070BD07
:106440003C780120747801200C4B1B6870B506461F
:106450000D4614460BB9FFF7B3FEF1B2084800F041
:106460000FFEE9B2064800F0EFFCE1B2044800F08C
:10647000EBFC0348BDE8704000F06DBE40780120A1
:10648000307901200128F8B536DD0D68EA0733D5EB
:106490001A4B4C681B686D100BB9FFF77DFEE9B213
:1064A000174800F0EDFD14F001050DD0C4F34701CD
:1064B000134800F0C9FC124800F04DFE18B123202B
:1064C000FBF770F80020F8BD042CF4D9236803F022
:1064D0000F03092BEFD154F8046F094F7610AE4229
:1064E000E9DD54F8041FCB0704D5C1F34701384652
:1064F00000F0AAFC0135F2E70120E4E73C78012036
:106500007478012038B50468E20702D54568EB07C6
:1065100004D40D20BDE83840FBF744B86410802C4B
:1065200001D91520F6E76D10FF2D01D91620F1E7EE
:10653000124B1B680BB9FFF72FFEE4B2214610483F
:1065400000F09EFDE9B20E4800F07EFC00210C48F0
:1065500000F0A0FD20B14042400040F0010038BDF5
:1065600001222146064800F088FD054800F063FC42
:106570000028F1D0024800F061FCEDE73C780120F2
:106580007478012038B5124B1B6804460D460BB9D0
:10659000FFF716FEE4B221460E4800F071FDE9B2A5
:1065A0000C4800F051FC0B4800F0D5FD08B140420A
:1065B00038BD01222146074800F05FFD054800F084
:1065C0003AFC0028F4D00348BDE8384000F036BC5F
:1065D0004078012030790120F8B5354E354D3768C7
:1065E00004466FB90D211D20FFF7CCFF5A2816D1A4
:1065F00001222A702A211D20FFF726FF0123336084
:1066000095F90030022B29D0032B44D0012B45D122
:1066100021461D20FFF7B6FF4FF0FF3424E00F2185
:106620001920FFF7AFFF332805D102232B705F221B
:1066300020211920E0E70D211E20FFF7A3FFC72826
:106640000AD103233A462A211E202B70FFF7FCFEB5
:106650001B222A211E20CFE72F70CFE7012C13D158
:1066600029211920FFF78EFF7F28C8BFA0F5807071
:106670006FF07E039842B8BF1846C82358437F2363
:1066800090FBF3F06043F8BD032C0BD12B211920B4
:10669000C0E72D21FBE721461E20BBE74FF0FF346A
:1066A0000020EAE7052CF4D04FF0FF340020DFE7AC
:1066B0004C7801202C00002008B50120FFF78CFF4A
:1066C000400040F0010008BD08B50320FFF784FF3B
:1066D000400040F0010008BD08B50520FFF77CFF31
:1066E000400040F0010008BD38B5104B1B6813B9DD
:1066F0000120FFF771FF0120FFF76EFF0446032022
:10670000FFF76AFF05460520FFF766FF6D4304FBB0
:10671000045400FB004002F03FFF01F09FFB03F038
:1067200055FA400040F0010038BD00BF4C78012010
:106730000128F8B535DD0F68FB0732D54D6815F037
:1067400001062ED1042D2CD92B6803F00F03092B41
:1067500027D16C68144B64101B68202CA8BF202420
:106760000BB9FFF719FDC7F3470122460F480F4F3A
:1067700000F083FC0435A64211DA0C4800F05BFB04
:1067800018B9700040F00100F8BD384600F056FB23
:10679000400040F0010045F8040F0136EBE76000CF
:1067A000F0E70120F0E700BF3C7801207478012079
:1067B000002070470120704700207047002070477C
:1067C000012070470020704700207047002070476C
:1067D000002070470020704700207047002070475D
:1067E00000207047002070477047704770470000D6
:1067F000024A03480E21FEF7ADBD00BF28C50000C8
:1068000098C500000246104601320378013B1F2B59
:10681000F9D9704708B5FFF7F5FF0378002B39D099
:10682000222B00F1010011D1037823B1222B00F1BA
:10683000010204D11046BDE80840FFF7E3BF5C2B1E
:1068400002D1437803B1821C1046EDE73A2BF2D017
:106850002C2BF0D07B2B0BD1FFF7D4FF0378002B30
:10686000E9D07D2B01D10130E5E7FFF7D3FFF5E754
:106870005B2B10D00246104612F8013B002BDAD0F9
:10688000202BD8DD2C2B05D003F0DF015D2901D0B2
:10689000222BF0D108BDFFF7B5FF0378002BCAD03B
:1068A0005D2BE0D0FFF7B6FFF7E708B5F0B1FFF7D3
:1068B000A9FF0378222B1AD07B2B1AD05B2B1AD07E
:1068C000A3F13002092A05D92D2B05D14278303A9F
:1068D000092A07D8032009E0742B0ED0662B0ED0AE
:1068E0006E2B0ED0181C18BF0120404208BD04209A
:1068F000FCE70220FAE70120F8E70520F6E706208A
:10690000F4E70720F2E738B5FFF77CFF03782D2B7B
:1069100011D101304FF0FF34431E00210A2501E060
:1069200005FB012113F8012F303AD0B20928F7D91D
:1069300004FB01F038BD0124EEE710B51446FFF763
:1069400061FF0378222B02D000230B7010BD621E62
:1069500001300378222BF7D0002BF5D05C2B07D029
:10696000441C002AF0DD01F8013B013A2046F0E723
:106970004378622B00F1020409D0662B09D06E2BFC
:1069800009D0722B09D0742B08BF0923E9E708232B
:10699000E7E70C23E5E70A23E3E70D23E1E710B57A
:1069A0000446FFF737FF0346A342184604D902788E
:1069B000202A03F1FF33F7D910BD08B590B1037851
:1069C00083B1FFF71FFF037803F0DF035D2B09D0CE
:1069D000FFF720FF03782C2B08BF0130BDE80840EB
:1069E000FFF710BF002008BD38B50D1E0DDD037880
:1069F0005B2B0AD10130FFF705FF0124A54205D02A
:106A0000FFF7DBFF10B10134F8E7002038BD38B5DF
:106A1000154609B100230B70F8B10378E3B1FFF715
:106A2000F1FE03782C2B044603D10130FFF7EAFE78
:106A3000044623787D2B0FD019B12A462046FFF754
:106A40007CFF2046FFF7E6FE03783A2B05D10130A4
:106A5000BDE83840FFF7D6BE002038BD2DE9F04133
:106A60000D469AB004462F789FB32E21284603F096
:106A7000EEFC804690B1461B303F092F13D82846C4
:106A8000FFF741FF01462046FFF7AEFF044604B37F
:106A9000B8F1000F1DD001363544E4E7284603F075
:106AA000EDFC0646E8E723787B2B11D1601C6422BD
:106AB00001A9FFF7ACFF044658B13246294601A8A8
:106AC00003F0E4FC0028E2D02046FFF7A3FEEEE747
:106AD000002420461AB0BDE8F08138B50D1E0446EA
:106AE0001CDDFFF7E2FE012807D1601C012D00D15B
:106AF00038BDFFF762FF013DF8E702280ED1002202
:106B00001146601CFFF783FF012DF1D0FFF755FF01
:106B100000221146FFF77BFF013DF5E70020E7E784
:106B2000F8B50C1E074615461E4613DDFFF7BDFEE1
:106B300002280FD132462946781CFFF768FF012C46
:106B400000D1F8BDFFF739FF32462946FFF75FFF56
:106B5000013CF4E70020F4E710B50446C8B1FFF7A4
:106B600051FE03787B2B0AD101300024002211460C
:106B7000FFF74DFF68B1FFF74DFE0134F6E75B2BE1
:106B800006D101300024FFF718FF10B10134FAE7F5
:106B90000024204610BD002870B514DD0D68EB07F9
:106BA00011D56D10013DFDF76BFE00264FF0FF344F
:106BB00060B916B3304603F061FC01463046BDE8CB
:106BC0007040FCF776BF4FF0FF35ECE70368C3F386
:106BD0000742152A0BD1C3F307239C42B8BF1C46BA
:106BE0009D4201D100F10806FDF74AFDE0E71D2AAC
:106BF00004BF00264FF0FF34F6E7601C400040F071
:106C0000010070BD10B508680C46FCF735FDFFF7B4
:106C100063F80028A2BF034B626843F820200020DD
:106C200010BD00BFC48B012008B50868FCF724FD27
:106C3000FFF752F80028AABF024B012053F82000AA
:106C400008BD00BFC48B012008B50868FCF714FD1F
:106C5000FFF742F80028ACBF0420002008BD000068
:106C6000024A03480421FEF775BB00BF28C6000096
:106C700021C6000008B5FCF731FCFCF7D1FCFEF79B
:106C80007DFB0448FEF787FDFDF73CFFBDE80840AB
:106C9000FEF760BE77C60000FCF7F0B838B50025F7
:106CA000057329B90B4B0C4A0C48232102F0B6FF9F
:106CB00001600B4951F82220027151F82330837191
:106CC0009DF8103051F8233043710223C371856061
:106CD00038BD00BF8FC60000EEC600009DC6000094
:106CE0004CC70000037B23B9437383730361012303
:106CF0000373704784B00DF1100C0CE90E009DF881
:106D00000810026800230129C2F80035039B12D045
:106D10000BD303290CD0C2F85435019BC2F824359B
:106D20000123C2F8003504B0704743F00203F2E7D4
:106D300043F00403EFE743F00603ECE710B5FFF779
:106D4000D1FF03688279C3F808254279C3F80C257E
:106D50000279C3F81025034BBDE810400ECBFFF7B6
:106D6000C9BF00BF687801200A0611D43F2912D894
:106D70001F2913D80F2914D8072915D803298CBF28
:106D80004FF080434FF000430268C2F8243570474B
:106D90004FF00073F8E74FF08063F5E74FF00063C2
:106DA000F2E74FF08053EFE74FF00053ECE7036852
:106DB000C3F81C15D3F80821002AFBD0D3F8180516
:106DC0000022C3F80821C0B27047000007B5094B84
:106DD00009490A484FF080421A6000229A60022254
:106DE0001A710F2300930E220D23FFF757FF03B0F4
:106DF0005DF804FB687801200030004054780120E1
:106E00002DE9F84380460D46174601EB02090C4672
:106E10004C45A4EB05060BD0D8F8003014F8011B44
:106E20001B68404698470028F2D13046BDE8F883F9
:106E30003E46FAE77047203000F03CBA203000F0C0
:106E40002BBA203000F03CBA38B5437F0D460BB961
:106E5000002038BD00F16804204600F039FA00280F
:106E6000F6D12046294600F008FA0120F1E700009B
:106E70002DE9F0411E4600254FF47A73C0E9015315
:106E80000C4B044640F8203B8846174600F0ECF9CE
:106E900004F1680000F0E8F99DF8183063769DF879
:106EA0001C302676C4E90487A37665772046BDE8C2
:106EB000F08100BF34C70000F0B5837E2E4C2F4D0B
:106EC0000121C17654F82320437E54F8233012F078
:106ED000200F14BF2F464FF0A04702F01F0213F0FF
:106EE000200F03F01F0308BF4FF0A04502F5E0722A
:106EF00003F5E07340F20C6647F8226045F8236022
:106F000003694FF0CC72C3F8242503690622C3F845
:106F10000025827E036954F82220C3F80825427EAA
:106F2000036954F82220C3F80C2590F91830144A4C
:106F30005C0903F01F03994004F1600342F8231039
:106F400090F91830002BBDBF03F00F0302F6FC329E
:106F5000D2189B18B5BF40234022137683F8002334
:106F600090F918300122590903F01F0302FA03F3C4
:106F7000034A42F82130F0BD4CC700000003005026
:106F800000E100E0C37EA3B103690022C3F800253D
:106F90000A4B99420ED90A4B994294BF4FF0806137
:106FA0004FF0C8610369C3F8241503690622C3F8CA
:106FB000002570474FF0CC71F4E700BFA0860100B8
:106FC00090D003002DE9F041044688461F4615463F
:106FD000002A50D000F12006304600F059F923690C
:106FE000C3F88885236901221A622369C3F83465CE
:106FF0002369C3F8385523691A602269D2F84C31E5
:107000001BB9D2F82431002BF8D00023C2F84C3140
:107010002269D2F85C311BB9D2F82431002BF8D0A8
:107020000023C2F85C3122696FB9D2F8243153B918
:107030000123D3612369D3F84821002AFBD0002221
:10704000C3F8482109E0012353612369D3F80421DF
:10705000002AFBD00022C3F804212369D3F824219D
:1070600012B10022C3F824212369D3F83C0520661D
:10707000C0B2BDE8F0811046FBE70123FFF7A2BFD5
:1070800010B5044680F8B010683000F001F9012313
:10709000637710BDF8B500234377036990F8B020FB
:1070A000C3F88825036901261E62036900F168059B
:1070B0000446C3F8445528460F4600F0FBF8236900
:1070C000C3F8480523699E602369D3F850211AB993
:1070D000D3F82421002AF8D00022C3F850212846F2
:1070E00000F0E8F8236930B1D3F860211AB9D3F879
:1070F0002421002AF8D00022C3F8602123696FB947
:10710000D3F8242152B90122DA612369D3F8482146
:10711000002AFBD00022C3F8482109E001225A616D
:107120002369D3F80421002AFBD00022C3F80421EC
:107130002369D3F8240168B10022C3F8242123690C
:10714000D3F8C404C3F8C404022803D004280CBF35
:1071500003200420F8BD0121FFF79CBF70B54369EF
:10716000D3F86421044692B10022012500F12006E3
:10717000C3F864210577304600F08AF86369C3F8E4
:10718000346563694022C3F8382563691D63636908
:10719000D3F86821DAB10025C3F8685104F1680614
:1071A000012363772577304600F072F8D4F8B430C5
:1071B00003B19847636965773046C3F8446500F0CA
:1071C00079F86369C3F84805636901225A63636902
:1071D000D3F8042162B10022C3F80421237F3BB11C
:1071E0006369D3F83C05D4F8B830206603B19847FA
:1071F0006369D3F8242152B10022C3F824216369C2
:10720000D3F8D024C3F8D024636901225A6170BD39
:107210000148FFF7A3BF00BF747801200148FFF7C2
:107220009DBF00BF3079012007B514231322CDE99B
:1072300000320A4A0A4811460323FFF719FE4FF0AD
:1072400040221E231F21CDE90031064804231146A8
:10725000FFF70EFE03B05DF804FB00BF00300040F6
:10726000747801203079012008B54022002102F015
:1072700067FD0022C0E9102208BD026C10B5531C46
:10728000446C03F03F039C421CBF8154036410BD57
:107290000023C0E910337047D0E9102393421FBF89
:1072A000C25C013303F03F03436414BF10464FF048
:1072B000FF307047D0E91030181A48BF403070478F
:1072C000D0E91023934214BFC05C4FF0FF307047E9
:1072D000036C406C013303F03F031B1A58425841C2
:1072E000704700000649074A074B9B1A03DD043B21
:1072F000C858D050FBDC00F04DF8F9F7A1F80000B9
:10730000F4CB00000000002034020020FEE7FEE77E
:10731000FEE7FEE7FEE7FEE7FEE7FEE7FEE7FEE745
:10732000094B1B78062B0CD1084B1B681A0708D198
:10733000074B186800F0F000A0F1300358425841A4
:1073400070470020704700BFE00F00F0E40F00F02E
:10735000E80F00F00C4B1B78062B10D10B4B1B6871
:107360001A070CD10A4B186800F0F003302B08D034
:1073700000F0E000A0F1400358425841704700205F
:1073800070470120704700BFE00F00F0E40F00F0ED
:10739000E80F00F008B5FFF7C3FF10B14A4B4B4AA6
:1073A0001A60FFF7D7FF28B1494B4A4A1B68C3F35D
:1073B00042331360FFF7B4FF20B1474AD36823F08C
:1073C0008073D360FFF7C6FF40B14FF080430022C7
:1073D000C3F80C21C3F81021C3F83825FFF7A0FF2C
:1073E00010B13E4B03221A60FFF79AFF40B13C4BAD
:1073F00005221A6001229A6700229A603F225A6091
:10740000384B1B78062B50D1374B1B681B074CD1D0
:10741000364B1B6803F0F003502B46D14FF08052DF
:10742000334BD2F80414C3F82015D2F80814C3F86B
:107430002415D2F80C14C3F82815D2F81014C3F888
:107440002C15D2F81414C3F83015D2F81814C3F858
:107450003415D2F81C14C3F84015D2F82014C3F820
:107460004415D2F82414C3F84815D2F82814C3F8E8
:107470004C15D2F82C14C3F85015D2F83014C3F8B8
:107480005415D2F83414C3F86015D2F83814C3F880
:107490006415D2F83C14C3F86815D2F84014C3F848
:1074A0006C15D2F84424C3F87025124AD2F88830FB
:1074B00043F47003C2F88830BFF34F8FBFF36F8F70
:1074C0000D4B0E4A1A6008BD74C007400DF0ADBAEE
:1074D000440200103C050040F0ED00E0A005004033
:1074E00010560040E00F00F0E40F00F0E80F00F04D
:1074F00000C0004000ED00E0300000200090D0030C
:107500000120704703681322DB691847704703693D
:10751000C3F81C150369D3F81C21002AFBD00022F4
:10752000C3F81C210120704710B490F95C30144C52
:1075300059090122203103F01F0302FA03F344F832
:10754000213003695DF8044B0421C3F80813036973
:107550005A600369DA6003690022C3F800250269F2
:107560004FF0FF33C2F80C350269C2F814350269D6
:10757000C2F8083502691430C2F81035FFF788BE2A
:1075800000E100E01430FFF795BE1430FFF798BE1D
:107590001430FFF781BE0000036990F85E2010B53B
:1075A000C3F80C25036990F85D20C3F8142590F802
:1075B00061200369012A01BF90F85F40C3F81045BC
:1075C000036990F8604006BFC3F8084503690022CC
:1075D000B1F5966FC3F86C2569D9B1F5166F69D905
:1075E000B1F5965F69D9B1F5165F68D9B1F5615FFC
:1075F00067D9B1F5964F66D9B1F5E14F65D9B1F5C7
:10760000164F64D9B1F5614F64D9B1F5963F64D98D
:10761000B1F5E13F63D9B1F5613F63D9364B99428A
:1076200063D9B1F5E12F63D9B1F5612F94BF4FF064
:1076300070634FF080530269C2F824350369042255
:10764000C3F8002501690023C1F808310169C1F8B8
:107650001C31016901230B6001698B600169C1F86C
:10766000042390F95C20510902F01F02934060311D
:10767000224A42F8213090F95C30002BBDBF03F064
:107680000F0302F6FC32D2189B18B5BF60236022AC
:10769000137683F8002390F95C300122590903F036
:1076A0001F0302FA03F3154A42F8213010BD4FF4CC
:1076B0009E23C0E74FF41D23BDE7114BBBE7114BE1
:1076C000B9E7114BB7E7114BB5E7114BB3E74FF4EF
:1076D0001D03B0E74FF46B03ADE70E4BABE74FF084
:1076E000EB73A8E74FF06C73A5E74FF08063A2E758
:1076F0004FF0E8639FE700BF90D0030000E100E097
:1077000000B013000050270000F03A0000A04E0027
:1077100000C0750000903A012DE9F0411E46002599
:107720004FF47A73C0E901530D4B044640F8143B03
:1077300017468846FFF798FD0A4AC4F8108084F877
:107740005C7052F8263084F85D309DF8183052F89D
:10775000233084F85E3084F861502046BDE8F08123
:10776000E0C700004CC7000010B50369D3F808213A
:1077700004464AB1D3F818151430C9B2FFF77DFD9D
:1077800023690022C3F8082110BD00000148FFF75B
:10779000EBBF00BFEC79012007B521230093022243
:1077A000222303490348FFF7B7FF03B05DF804FB4A
:1077B00000200040EC79012008B102F08DBD704737
:1077C0000A4B19680A4B30B5D3F804050C060D0AAC
:1077D00044EA00024FF47A712B46A2FB014501FBFB
:1077E0000355E00B40EA454030BD00BF507A012010
:1077F0000010014038B5044648B1FFF7E1FF0546E7
:1078000000F01AF8FFF7DCFF401BA042F8D338BDA8
:10781000074B0022C3F8042182B0D3F80431054A93
:107820000193019B13680133DBB2136002B0704710
:1078300000100140507A01207047704708B500F0F1
:107840005FF8FFF7FAFF0120FFF7D4FFFFF712FA06
:10785000034CFFF721FA002CFBD0AFF30080F8E7D0
:1078600000000000134B53F8203010B503F01F0345
:10787000114C0120002900FA03F010492368B3FBE2
:10788000F1F3014602FB03F34FF00A02B3FBF2F3FC
:1078900014BF024600220A4800F014F842F21073A6
:1078A00058434FF47A722368B3FBF2F3B0FBF3F062
:1078B00010BD00BF4CC700003000002040420F0048
:1078C0001005005030B504680C40944206D1013BCD
:1078D000002BF8D112E0013B002B0FD004680C40C4
:1078E0009442F8D1002405680D40954204D101343A
:1078F0009C42F8D1002002E0201C00E0181C30BDA2
:107900000D4BE02283F811234FF40032C3F880219D
:107910001A604FF080430122C3F818259A6003F5DE
:1079200088330021C3F808150221C3F80413C3F8F3
:1079300044131A60704700BF00E100E0014B18607B
:10794000704700BF48000020222837B50CD84B4BA9
:1079500053F82030052B00F0828007D8032B12D07B
:107960007BD8022B00F08180002074E01D2B78D0A2
:1079700003D81C2BF8D1052206E01E2B73D01F2B39
:10798000F2D1082200E002223D4B196808296EDD81
:107990000A296FDD0D29B5BF0C240E240223032311
:1079A0003848C0F8F0350123C0F8003500200546FE
:1079B000030103F1804303F5E04301300828C3F8D5
:1079C0001455C3F81055F3D12F4B18682F4B1B6873
:1079D00000021B0303F4805300F4E0601843294BBA
:1079E000C3F81805C3F81425C3F810250DF10602D5
:1079F000C3F82C260122C3F830261A60D3F80021E0
:107A0000002AFBD00022C3F8002101225A601D4B3E
:107A10001A46D3F804010028FBD00020C3F8040163
:107A200001209860D2F81431002BFBD00023C2F85B
:107A30001431BDF906209A42124AB8BFADF806309B
:107A4000A142C2F80035BDF9060004D035BF611A65
:107A5000091BC840884003B030BD032294E70422CC
:107A600092E7062290E707228EE701228CE708249E
:107A7000002395E70A24012392E700BF4CC70000CA
:107A80004000002000700040440000205C7A01208B
:107A9000222830B53CD8224B53F82000214B00223D
:107AA0001D4653F82240B4F1FF3F32D11E4C45F839
:107AB00022006FEA41411D4D1D4B246853F82230CE
:107AC0006FEA514125F81210012101FA04F4C3F8BC
:107AD0006005013CC3F8640505EB4202C3F8680584
:107AE000C3F86C050020C3F80015C3F80C05C3F8F3
:107AF0000405C3F80845C3F81405C3F81005C3F816
:107B00002025C3F82415C3F82815C3F82C0599605F
:107B100030BD8442CAD00132032AC2D1F8E700BF87
:107B20004CC700003400002048000020547A012097
:107B300008C80000222815D8114B124A53F82030EB
:107B400013F0200F08BF4FF0A04203F01F030329DA
:107B500008D8DFE801F00210080C03F5E0730021FB
:107B600042F82310704703F5E0730C21F8E703F5A2
:107B7000E0730421F4E703F5E0730321F0E700BFAD
:107B80004CC7000000030050222813D80A4B53F8BA
:107B900020000A4B10F0200F4FF0010200F01F00F0
:107BA00008BF4FF0A043824011B9C3F80C257047BD
:107BB000C3F80825704700BF4CC700000003005001
:107BC000222810D8094B0A4A53F8203013F0200F0E
:107BD00008BF4FF0A04203F01F03D2F81005D840B1
:107BE00000F0010070470020704700BF4CC7000044
:107BF000000300502DE9F04106460D4601EB020856
:107C00000C464445A4EB050707D0336814F8011B64
:107C10001B68304698470028F3D13846BDE8F0810C
:107C20002DE9F041C1F30A57A7F2FF35132D82B0B9
:107C300002460B460C464FEAD178064633DC002D4F
:107C40004EDB3B49294103EA0100104326D0490895
:107C50000B4052EA03060CD04FF48023132D24EA84
:107C6000010143FA05F444EA01040CBF4FF0004659
:107C70000026304901EBC8082346D8E900453246C2
:107C80002046294601F03CFBCDE9000122462B4667
:107C9000DDE9000101F032FB02460B4610461946B1
:107CA00002B0BDE8F081332D07DDB5F5806FF5D169
:107CB00001F026FB02460B46F0E7A7F213474FF010
:107CC000FF31F9400842E9D049080842D1D04FF0CD
:107CD000804320EA010143FA07F741EA0706C8E7B3
:107CE00021F000410143D9D0C3F3130101434E42B7
:107CF000104D0E43360B05EBC8055C0C06F4002353
:107D0000D5E90067640443EA04010B46304639466E
:107D100001F0F6FACDE9000132463B46DDE900010B
:107D200001F0ECFA21F00041024641EAC873B5E7E0
:107D3000FFFF0F0018C80000F8B5C1F30A57A7F2FB
:107D4000FF35132D0A460B46044611DC002D2ADBB5
:107D50008C461F4929410A422BD04FF400232B4166
:107D6000634423EA01030026344619462046F8BD41
:107D7000332D05DDB5F5806F1ED011462046F8BDC8
:107D8000A7F213474FF0FF3121FA07F73842F4D03A
:107D90000122C5F1330502FA05F5461928BF9B18E3
:107DA00026EA0706E0E7013501F0004309D0002686
:107DB000DAE70028D1D1E0E7024601F0A1FA044653
:107DC000DCE743F07F5343F440130026CCE700BFC9
:107DD000FFFF0F0030B51F4A21F00043934287B0E8
:107DE0001BDD1D4A934205DD02460B4601F086FA73
:107DF00007B030BD02AA00F08FF800F003000128A0
:107E0000DDE9042311D002281BD098B1DDE902017D
:107E100000F062FB01F10041EAE700230093002239
:107E2000002301F09DF807B030BDDDE9020100F04C
:107E300053FBDDE70124DDE90201009401F090F835
:107E4000D6E70124DDE90201009401F089F801F18F
:107E50000041CDE7FB21E93FFFFFEF7F2DE9F04F28
:107E60008BB004460D4600F075FA294B93F900A03B
:107E7000BAF1FF3F06460F4612D022462B46204657
:107E8000294601F08DFE834650B94FF000084FF0AF
:107E9000000942464B462046294601F059FE20B9CA
:107EA000304639460BB0BDE8F08F0122194BCDF8B2
:107EB00020B00092CDE90445CDE902450193BAF125
:107EC000000F17D042464B464046494601F0F8FCA9
:107ED000BAF1020FCDE906010ED101F0BDFE21235A
:107EE0000360089B73B9DDE90667304639460BB07D
:107EF000BDE8F08FCDE90689684601F071F90028E8
:107F0000EFD1EAE701F0A8FE089B0360EBE700BFB2
:107F10004C00002028C800002DE9F04FC84E21F089
:107F20000047B7428FB00B4640F38F809246C54A58
:107F300097420C4626DC0029B7A3D3E9002340F37F
:107F40008F8001F0DBF9C04B9F4204460D4600F0E4
:107F50004681B3A3D3E9002301F0D0F902460B46D2
:107F6000CAE900232046294601F0C8F9ACA3D3E9A9
:107F7000002301F0C3F90125CAE9020128460FB028
:107F8000BDE8F08FB14A974240F38980B04A9742EA
:107F900000F31C813D15A5F21645A7EB05531946C4
:107FA0001F46064601F012FE01F0F6FA80468946A9
:107FB00002460B4630463946CDE9088901F09EF964
:107FC0000022A44B01F052FB8946804601F0FEFDE1
:107FD00001F0E2FA02460B4606460F464046494685
:107FE000CDE90A6701F08AF900229A4B01F03EFBC5
:107FF00000220023CDE90C0101F0A0FD002800F0D3
:108000005D81002330463946002201F097FD0028AB
:1080100014BF01230223904A019202212A460091B3
:1080200008A8514600F07CFB002C054614DADAF86B
:108030000420DAF80C3002F1004203F1004345421B
:10804000CAF80420CAF80C3006E0C2E90001002595
:108050000024C2E90245002528460FB0BDE8F08F94
:1080600001F04EF9784B9F4204460D4600F008811E
:108070006BA3D3E9002301F043F902460B46CAE99A
:1080800000232946204601F039F965A3D3E90023EE
:1080900001F036F94FF0FF35CAE90201DCE701F0E3
:1080A00015F861A3D3E900238046894601F0DEFA82
:1080B00000226A4B01F024F901F088FD054601F029
:1080C0006BFA55A3D3E90023CDE9040101F0CEFA00
:1080D00002460B464046494601F010F950A3D3E949
:1080E0000023CDE90201DDE9040101F0BFFA1F2DF3
:1080F0008046894602460B46DDE9020140F3B08026
:1081000001F0FCF883460E463F15C6F30A53FB1AEE
:10811000102B40F3B08046A3D3E90023DDE904012E
:1081200001F0A4FA8046894602460B46DDE90201C9
:1081300001F0E4F802460B46DDE90201CDE9062331
:1081400001F0DCF842464B4601F0D8F83AA3D3E9F7
:10815000002380468946DDE9040101F087FA4246A2
:108160004B4601F0CBF80B46024680468946DDE9D6
:10817000060101F0C3F8C1F30A53FF1A312F8346F9
:108180000E4600F39D8002460B46CAE90023DDE956
:108190000623CDE902235A463346DDE9020101F008
:1081A000ADF842464B4601F0A9F8002C02460B46BA
:1081B000CAE90223BFF650AF06F1004601F10041C3
:1081C000CAE900B6CAE902016D4245E7024601F07C
:1081D00095F80025CAE90201CAE900013CE714A3A9
:1081E000D3E9002301F08AF813A3D3E900230D4655
:1081F000044601F083F802460B46CAE900232946EB
:10820000204601F07BF80CA3D3E9002301F076F8B7
:108210000125CAE902011FE700004054FB21F93F94
:108220003163621A61B4D03D83C8C96D305FE43FE9
:108230000000601A61B4D03D7370032E8A19A33B0D
:10824000FB21E93F7BD90240FB21F93FFB2139416A
:10825000FFFFEF7F00007041B0C800000000E03F6A
:1082600001F04CF83A4B6A1E834653F82230BB4269
:108270000E463FF449AF5A463346CAE900238AE71F
:108280002BA3D3E9002301F03BF82BA3D3E9002370
:108290000D46044601F034F802460B46CAE90023B5
:1082A0002946204601F02AF823A3D3E9002301F050
:1082B00027F84FF0FF35CAE90201CDE60323AAE60D
:1082C0001FA3D3E90023DDE9040101F0CFF9DDE9C3
:1082D000068906460F4602460B464046494601F0CF
:1082E0000DF802460B4640464946CDE9022301F00F
:1082F00005F832463B4601F001F813A3D3E9002309
:1083000006460F46DDE9040101F0B0F932463B466E
:1083100000F0F4FF02460B4680468946DDE9020183
:1083200000F0ECFF83460E46A5E700BFAFF30080E8
:108330000000601A61B4D03D7370032E8A19A33B0C
:108340000000002E8A19A33BC14920259A837B395E
:1083500030C800005F4A8A432DE9F0410D460746C8
:1083600000F0948000290B460446064654DD0F15A4
:1083700000F0A780C3F31303A7F2FF3743F4801381
:10838000F20FF80702EB43034FEA460503D5ED0F62
:1083900005EB4303B50000267F10B44616224FF4C8
:1083A00000110CEB010098424FEAD5744FEA4505E5
:1083B00003DC1B1A00EB010C0E44013A04EB4303EF
:1083C0004FEA5101EDD11046964620244FF000426D
:1083D00009E052D05B00013C03EBD5734FEA520237
:1083E0004FEA450537D0634502EB0E01F1DD002968
:1083F00001EB020E0ADBE046A3EB0C03A94288BFA7
:1084000003F1FF336D1A1044C446E3E7BEF1000FD9
:10841000F1DB0CF10108EFE721F00042024329D023
:10842000002945D10146CA0A153B4905002AFAD060
:1084300012F4801001D048E030465200D40200F11E
:108440000106F9D5C6F1200401FA06F6E1401F1A2B
:1084500041EA02038EE72B4324D14408731003F151
:108460007F53F20703F5001348BF44F0004403EBC9
:10847000075127463846BDE8F081A942AAD800290D
:1084800001EB020EC2DB98460023BBE702460B4617
:1084900001F0ECF83A462B4600F032FF074638462A
:1084A000BDE8F081411C16BF421C01365408D5E7D7
:1084B000024600F023FF02460B4601F001FA074690
:1084C000D8E71A4621463B46B2E70E4620244FF035
:1084D000FF30BBE70000F07F2DE9F04F21F00046B0
:1084E000B6F1795F85B00C4692469B4605466BDA3D
:1084F00001F06CFB002800F0E2802A462346284663
:10850000214601F0B3F874A3D3E9002380468946DD
:1085100001F0ACF872A3D3E9002300F0F1FE42466B
:108520004B4601F0A3F870A3D3E9002300F0E6FE68
:1085300042464B4601F09AF86DA3D3E9002300F0C0
:10854000DFFE42464B4601F091F86BA3D3E90023CE
:1085500000F0D4FE42464B4601F088F868A3D3E908
:10856000002300F0CDFE42464B4601F07FF8CDE9F6
:1085700000010022644B4046494601F077F8DDE9EE
:10858000002306460F464046494601F06FF8524622
:10859000804689465B462846214601F067F8024638
:1085A0000B464046494600F0A9FE02460B463046BF
:1085B000394600F0A3FE02460B460020534900F066
:1085C0009DFE05B0BDE8F08F02460B4601F04EF867
:1085D00041A3D3E900238046894601F047F840A330
:1085E000D3E9002300F08CFE42464B4601F03EF8F2
:1085F0003DA3D3E9002300F081FE42464B4601F043
:1086000035F83BA3D3E9002300F07AFE42464B46FF
:1086100001F02CF838A3D3E9002300F06FFE4246A6
:108620004B4601F023F836A3D3E9002300F068FE9F
:108630004B46424601F01AF8354B9E42CDE9000107
:1086400097DD344B9E424FF000023DDCA6F500134F
:1086500000202E4916461F4600F050FECDE90201CB
:108660000022294B4046494601F000F832463B467D
:1086700000F044FEDDE9002306460F464046494629
:1086800000F0F4FF5246804689465B462846214664
:1086900000F0ECFF02460B464046494600F02EFE35
:1086A00002460B463046394600F028FE02460B468D
:1086B000DDE9020100F022FE05B0BDE8F08F1349AC
:1086C000002005B0BDE8F08F134B144FCDE9022315
:1086D0000026C5E7AFF30080D43888BEE9FAA8BD0C
:1086E000C4B1B4BD9EEE213EAD529C804F7E923E01
:1086F0009015CB19A001FA3E7751C1166CC1563FB7
:108700004C5555555555A53F0000E03F0000F03F42
:108710003233D33F0000E93F0000E73F0000D23F83
:108720002DE9F04FADF5197DBE4CA29EBE4D54F81B
:1087300026700793D41E85FB0465E417C4EBA504DB
:1087400024EAE4741D46631CA3EB8303013D02EBA2
:10875000C30305937B1909940497019506460B9171
:10876000A4EB05041BD423445D1C20AF4FF000088C
:108770004FF00009DDF88CA208E05AF8240000F060
:108780000BFF0134AC42E7E8020108D0002CF4DA18
:10879000013440464946AC42E7E80201F6D1049B69
:1087A000002BC0F2B083079BA6F10802DB00114644
:1087B000039220AA02EB0309029301EB0308049B36
:1087C00072AA02EBC30B0DF5E07A019B002BC0F2FD
:1087D0009581039C4D460026002775E90223F4E9A4
:1087E000020100F043FF02460B463046394600F0D6
:1087F00087FD444506460F46EFD1EAE80267DA45B1
:1088000009F10809E1D1DDE90204049920448B0053
:1088100082460BA8A3F10802C31808930CAB1344BB
:108820000A938B4698AB03EBCB03BBF1000F53E9E4
:10883000284529DD70AB03EBCB080DF13009002290
:108840007A4B2046294600F011FF01F0BFF900F0F5
:10885000A3FE0022764B06460F4600F007FF0246B5
:108860000B462046294600F049FD01F0AFF978E9B2
:10887000022349F8040B3946304600F041FD70AB45
:10888000984504460D46DAD1DDF814902046294675
:108890004A4600F0A9FC00224FF07F5304460D46E3
:1088A00000F0E4FE00F018FC0022624B00F0DEFE57
:1088B00002460B462046294600F020FD0D460446A0
:1088C00001F084F9804600F067FE0B460246294617
:1088D000204600F013FD4B46002B06460F4640F3A2
:1088E000E1800BF1FF320CA9C9F1180351F82250B5
:1088F00045FA03F101FA03F30CA8EB1A40F8223011
:10890000C9F11705884443FA05F5002D2CDDBBF1AC
:10891000000F08F1010840F394820C9C002C40F0F9
:10892000A780BBF1010F0AD00CA9012251F8044F16
:10893000531C002C40F09E809B451A46F6D1059BA7
:10894000002B0EDD012B00F09C81022B09D10BF1D5
:10895000FF320CAB0CA953F82230C3F3150341F8D6
:108960002230022D00F0AF8000220023304639462D
:1089700001F0E4F8002800F06682049B0BF1FF3957
:108980004B4510DC0BF180430CAA013B089802EB2D
:108990008303002253F80419834242EA0102F9D109
:1089A000002A40F0B580049B0CAA013B52F823300A
:1089B000002B40F0A1800A9A012352F804190133D8
:1089C0000029FAD05B440BF101099945069349DC73
:1089D000099A079909EB020801EB0B0508F1804899
:1089E00002EB030BA39B08F1FF3803EB880870AB85
:1089F00003EBC909A39B20A903EB8B0301EBC5057E
:108A0000029358F8040F00F0C7FD019B002BC5E945
:108A1000000105F1080B28DB083D039C0026002718
:108A20000CE000BFF8C90000ABAAAA2A0000703E03
:108A3000000070410000204075E80201F4E90223C3
:108A400000F014FE02460B463046394600F058FC52
:108A5000544506460F46EFD1029B9845E9E8026768
:108A60005D46CED1DDF818B0DCE600260027F3E73E
:108A7000012300220CA9C4F180749B4541F82240D7
:108A80000EDD51F8232001EB8B0001EB83036FF027
:108A90007F4100E01A688A1A43F8042B8342F9D117
:108AA00001244CE706D10BF1FF330CAA52F82350F6
:108AB000ED152AE70022BE4B01F05EF8002840F0D9
:108AC000B981054650E732463B460020B94900F0DF
:108AD00015FC06460F46002C3FF446AF059AB549F3
:108AE000002000F081FB02460B463046394600F07C
:108AF00005FC06460F4637E7012363E700260027FB
:108B0000EAE80267DA4509F108097FF45EAE7AE621
:108B10000CAB059A53F82930183ACDE90685059231
:108B20006BB909F18043013B0CA901EB830353F8B6
:108B3000041909F1FF39183A0029F8D00592059A6D
:108B40009C49002000F050FBB9F1000F04460D468F
:108B5000C0F2E0814FEAC90370AA02EB0308089350
:108B60000CAB03EB8906DFF850B208F108070436B6
:108B70004FF0000A56F8040D00F00EFD22462B4679
:108B800000F074FD5B4667E9020152462046294623
:108B900000F06CFD0CAB9E4204460D46EAD148AB9A
:108BA00003930193CDF8149009F10103DDF81090BF
:108BB0000293C3464FF0000AB9F1000FC0F23781AB
:108BC000DFF8F8815D4678A3D3E90023002600276B
:108BD000002403E0544510DCF8E80223F5E8020124
:108BE00000F044FD02460B463046394600F088FB53
:108BF0000134A14506460F46ECDA019BE3E8026723
:108C00000193029B0AF1010A9A45ABF1080BD3D1FB
:108C1000A29BDDF81490032B2CD8DFE813F0E800BA
:108C2000D300D3003F00079B00200146002B40F0FB
:108C300043810D460B460B990446C1E90045039953
:108C40000246D1E9000100F059FBB9F1000F0CDD3B
:108C5000039D0124F5E90223013400F051FBA145F5
:108C6000F8DA079B002B40F037810B460B99024640
:108C7000C1E90223069B03F007000DF5197DBDE84D
:108C8000F08F0BF1FF320CAB0CA953F82230C3F379
:108C9000160341F8223064E648AB0393B9F1000FA4
:108CA00040F35581039ACDF808904FEAC90302EBCF
:108CB0000308D8E900AB0193914658E90267524690
:108CC0005B463046394600F01BFB04460D46024623
:108CD0000B463046394600F011FB52465B4600F029
:108CE0000FFBC8E9000168E90245C145A246AB4651
:108CF000E3D1DDF80890B9F1010F40F32881019B21
:108D0000039A1344D3E9006701939A460DF5947BC7
:108D10005AE9028932463B464046494600F0F0FA9D
:108D200004460D4602460B464046494600F0E6FA28
:108D300032463B4600F0E4FACAE900016AE902451E
:108D4000D34526462F46E3D10399019C002301F128
:108D50001005083419461E46304674E9022300F017
:108D6000CFFAA5420346F6D10A460399D1E9008C11
:108D7000D1E902E90799002900F0B1800B9C236139
:108D8000069BC4F800800CF1004009F1004102F19B
:108D90000042606003F00700E1606261C4F808E02F
:108DA0000DF5197DBDE8F08F00000040FB21F93F73
:108DB0000000E03F0000F03F0000703EC0C900002E
:108DC00048AB0393B9F1000FFFF62DAF039F0020CE
:108DD00007EBC9060836014676E9022300F090FA4F
:108DE000B742F9D1079B002B3FF423AF64E0089C06
:108DF000039D083400222C4411461646304674E97F
:108E0000022300F07DFAA5420246F6D10B460799EF
:108E100009B103F1004319460B9B1046C3E9000159
:108E2000069B03F007000DF5197DBDE8F08F0026C5
:108E30000027E2E6BBF1000F08F101087DDD022505
:108E40006BE500247BE5CDE90685059D3046394676
:108E50006A4200F0C9F900223E4B06460F4600F078
:108E60008BFE00B300223C4B3046394600F0FEFB3F
:108E700000F0ACFE044600F08FFB0022354B00F002
:108E8000F5FB0B4602463946304600F037FA00F053
:108E90009DFE0BF101090CAB183543F82B0005952D
:108EA00043F829404BE63046394600F08FFE0CABC4
:108EB000D94643F82B0042E60B9C0B4601F10041DA
:108EC000C4E9000103990246D1E9000100F016FA55
:108ED000B9F1000F3FF7BCAE01F10041C5E61846FD
:108EE0000B9B4646744667464D461146C3E904014E
:108EF000C3E90067C3E90245069B03F007000DF5CF
:108F0000197DBDE8F08FA6F108030393079BDB00F2
:108F1000029378E4A29B032B3FF6ACAE01A252F879
:108F200023F000BF358F0000C18D0000C18D00000F
:108F3000998C00000022134669E732463B46002028
:108F4000064900F0DBF9022506460F460CE5002332
:108F50001A460AE7000070410000703E0000F03F32
:108F60002DE9F04F21F00046B6F1795F85B00C464F
:108F700090469946054604DA00F028FE002800F0E5
:108F800085802A4623462846214600F06FFB064688
:108F90000F4602460B462846214600F067FB3EA3DB
:108FA000D3E9002382468B463046394600F05EFB0B
:108FB0003BA3D3E9002300F0A1F932463B4600F081
:108FC00055FB39A3D3E9002300F09AF932463B461A
:108FD00000F04CFB36A3D3E9002300F08FF93246B2
:108FE0003B4600F043FB34A3D3E9002300F088F9AB
:108FF0000E9BCDE900019BB30022334B404649460E
:1090000000F034FBDDE90023CDE90201504659466A
:1090100000F02CFB02460B46DDE9020100F06EF980
:1090200032463B4600F022FB42464B4600F066F9D2
:1090300023A3D3E9002306460F465046594600F0C5
:1090400015FB02460B463046394600F059F90246F8
:109050000B462846214600F051F905B0BDE8F08FD7
:1090600002460B463046394600F000FB14A3D3E914
:10907000002300F043F952465B4600F0F7FA2A4617
:10908000234600F03DF905B0BDE8F08F28462146A3
:1090900005B0BDE8F08F00BF7CD5CF5A3AD9E53D89
:1090A000EB9C2B8AE6E55A3E7DFEB157E31DC73E99
:1090B000D561C119A0012A3FA6F810111111813FF5
:1090C000495555555555C53F0000E03F21F0004337
:1090D0001946704700000000C1F30A522DE9F84319
:1090E000A2F2FF36132E0B460D460446884607466D
:1090F0001DDC002E3DDB384A42FA06F901EA09027E
:10910000024319D032A3D3E9002300F0F9F800227A
:10911000002300F03BFDD0B3002D04DA4FF48013A0
:1091200043FA06F6B04428EA090500272FE0332E5B
:1091300006DDB6F5806F2FD019462046BDE8F883CE
:10914000A2F213424FF0FF3929FA02F919EA000F8F
:10915000F2D01FA3D3E9002300F0D2F800220023AD
:1091600000F014FD98B1002D24DB27EA09074546DD
:109170000DE017A3D3E9002300F0C2F8002200237A
:1091800000F004FD18B1002D0BDB00273D463C46E6
:1091900029462046BDE8F883024600F0B1F80446AF
:1091A000CBE725F000430D4A1F43002F18BF15469B
:1091B0000027ECE7142E08D00123C6F1340603FA89
:1091C00006F6371928BF9844CFE705F10108CCE728
:1091D0009C7500883CE4377EFFFF0F000000F0BF65
:1091E0000020704700000000F8B5C1F30A530446A0
:1091F0000D460E4617460BBB21F00046034633438F
:109200001BD0354B002200F031FA344B9F4204460C
:109210000D4635DBC1F30A530E46363B3B4440F264
:10922000FE72934232DC002B11DD26F0FF4626F45D
:10923000E00646EA035520462946F8BD40F2FF7293
:109240009342EBD102460B4600F05AF8F8BD13F1F9
:10925000350F28DA4CF250339F4222462B460ADD66
:1092600019A1D1E9000100F03DF817A3D3E90023CB
:1092700000F0FCF9F8BD16A1D1E9000100F032F8C8
:1092800013A3D3E9002300F0F1F9F8BD22462B46E1
:109290000DA1D1E9000100F025F80BA3D3E90023CB
:1092A00000F0E4F9F8BD26F0FF4626F4E006363378
:1092B00046EA0355204629460022094B00F0D6F91C
:1092C000F8BD00BFAFF300809C7500883CE4377E9A
:1092D00059F3F8C21F6EA50100005043B03CFFFFD8
:1092E0000000903C03F0004321F0004242EA0301F9
:1092F000704700BF81F0004102E000BF83F00043EF
:1093000030B54FEA41044FEA430594EA050F08BF20
:1093100090EA020F1FBF54EA000C55EA020C7FEAE4
:10932000645C7FEA655C00F0E2804FEA5454D4EB61
:109330005555B8BF6D420CDD2C4480EA020281EA2B
:10934000030382EA000083EA010180EA020281EA63
:109350000303362D88BF30BD11F0004F4FEA0131B5
:109360004FF4801C4CEA113102D0404261EB4101C4
:1093700013F0004F4FEA03334CEA133302D052424A
:1093800063EB430394EA050F00F0A780A4F1010406
:10939000D5F1200E0DDB02FA0EFC22FA05F2801840
:1093A00041F1000103FA0EF2801843FA05F3594126
:1093B0000EE0A5F120050EF1200E012A03FA0EFCA5
:1093C00028BF4CF0020C43FA05F3C01851EBE371CF
:1093D00001F0004507D54FF0000EDCF1000C7EEBEC
:1093E00000006EEB0101B1F5801F1BD3B1F5001F2A
:1093F0000CD349085FEA30004FEA3C0C04F1010449
:109400004FEA445212F5800F80F09A80BCF1004F71
:1094100008BF5FEA500C50F1000041EB045141EAF3
:10942000050130BD5FEA4C0C404141EB010111F4F4
:10943000801FA4F10104E9D191F0000F04BF01469F
:109440000020B1FA81F308BF2033A3F10B03B3F17D
:1094500020020CDA0C3208DD02F1140CC2F10C020D
:1094600001FA0CF021FA02F10CE002F11402D8BF6B
:10947000C2F1200C01FA02F120FA0CFCDCBF41EA37
:109480000C019040E41AA2BF01EB0451294330BD06
:109490006FEA04041F3C1CDA0C340EDC04F11404E3
:1094A000C4F1200220FA04F001FA02F340EA0300BA
:1094B00021FA04F345EA030130BDC4F10C04C4F100
:1094C000200220FA02F001FA04F340EA03002946E0
:1094D00030BD21FA04F0294630BD94F0000F83F42A
:1094E000801306BF81F480110134013D4EE77FEA0D
:1094F000645C18BF7FEA655C29D094EA050F08BF59
:1095000090EA020F05D054EA000C04BF1946104639
:1095100030BD91EA030F1EBF0021002030BD5FEA7D
:10952000545C05D14000494128BF41F0004130BDA5
:1095300014F580043CBF01F5801130BD01F00045F9
:1095400045F0FE4141F470014FF0000030BD7FEA6C
:10955000645C1ABF194610467FEA655C1CBF0B4667
:10956000024650EA013406BF52EA033591EA030F7E
:1095700041F4002130BD00BF90F0000F04BF002176
:10958000704730B54FF4806404F132044FF00005A9
:109590004FF0000150E700BF90F0000F04BF002122
:1095A000704730B54FF4806404F1320410F0004588
:1095B00048BF40424FF000013EE700BF42004FEA83
:1095C000E2014FEA31014FEA02701FBF12F07F4300
:1095D00093F07F4F81F06051704732F07F4208BFB7
:1095E000704793F07F4F04BF41F40021704730B5BE
:1095F0004FF4607401F0004521F000411CE700BF0A
:1096000050EA010208BF704730B54FF000050AE08C
:1096100050EA010208BF704730B511F0004502D58D
:10962000404261EB41014FF4806404F132045FEA8F
:10963000915C3FF4D8AE4FF003025FEADC0C18BF38
:1096400003325FEADC0C18BF033202EBDC02C2F12A
:10965000200300FA03FC20FA02F001FA03FE40EABC
:109660000E0021FA02F11444BDE600BF70B54FF0C0
:10967000FF0C4CF4E06C1CEA11541DBF1CEA13559E
:1096800094EA0C0F95EA0C0F00F0DEF82C4481EA06
:10969000030621EA4C5123EA4C5350EA013518BF26
:1096A00052EA033541F4801143F4801338D0A0FB13
:1096B00002CE4FF00005E1FB02E506F00042E0FBC0
:1096C00003E54FF00006E1FB03569CF0000F18BFC6
:1096D0004EF0010EA4F1FF04B6F5007F64F540746E
:1096E00004D25FEA4E0E6D4146EB060642EAC62101
:1096F00041EA55514FEAC52040EA5E504FEACE2E6E
:10970000B4F1FD0C88BFBCF5E06F1ED8BEF1004F70
:1097100008BF5FEA500E50F1000041EB045170BDEC
:1097200006F0004646EA010140EA020081EA030130
:10973000B4EB5C04C2BFD4EB0C0541EA045170BD2C
:1097400041F480114FF0000E013C00F3AB8014F1A6
:10975000360FDEBF002001F0004170BDC4F10004EF
:10976000203C35DA0C341BDC04F11404C4F1200570
:1097700000FA05F320FA04F001FA05F240EA0200CB
:1097800001F0004221F0004110EBD37021FA04F601
:1097900042EB06015EEA430E08BF20EAD37070BDBB
:1097A000C4F10C04C4F1200500FA04F320FA05F01A
:1097B00001FA04F240EA020001F0004110EBD3701C
:1097C00041F100015EEA430E08BF20EAD37070BD8C
:1097D000C4F1200500FA05F24EEA020E20FA04F365
:1097E00001FA05F243EA020321FA04F001F0004114
:1097F00021FA04F220EA020000EBD3705EEA430E85
:1098000008BF20EAD37070BD94F0000F0FD101F0B3
:109810000046400041EB010111F4801F08BF013CEC
:10982000F7D041EA060195F0000F18BF704703F02A
:109830000046520043EB030313F4801F08BF013DB1
:10984000F7D043EA0603704794EA0C0F0CEA13556D
:1098500018BF95EA0C0F0CD050EA410618BF52EA27
:109860004306D1D181EA030101F000414FF000002D
:1098700070BD50EA410606BF1046194652EA43063B
:1098800019D094EA0C0F02D150EA013613D195EAAF
:109890000C0F05D152EA03361CBF104619460AD1F7
:1098A00081EA030101F0004141F0FE4141F4700101
:1098B0004FF0000070BD41F0FE4141F4780170BDF1
:1098C00070B54FF0FF0C4CF4E06C1CEA11541DBF56
:1098D0001CEA135594EA0C0F95EA0C0F00F0A7F858
:1098E000A4EB050481EA030E52EA03354FEA013185
:1098F00000F088804FEA03334FF0805545EA131398
:1099000043EA12634FEA022245EA111545EA10655F
:109910004FEA00260EF000419D4208BF964244F1F6
:10992000FD0404F5407402D25B084FEA3202B61A15
:1099300065EB03055B084FEA32024FF480104FF4E9
:10994000002CB6EB020E75EB030E22BFB61A75465D
:1099500040EA0C005B084FEA3202B6EB020E75EBF0
:10996000030E22BFB61A754640EA5C005B084FEA58
:109970003202B6EB020E75EB030E22BFB61A754625
:1099800040EA9C005B084FEA3202B6EB020E75EB30
:10999000030E22BFB61A754640EADC0055EA060EF1
:1099A00018D04FEA051545EA16754FEA06164FEA34
:1099B000C30343EA52734FEAC2025FEA1C1CC0D1E0
:1099C00011F4801F0BD141EA00014FF000004FF06D
:1099D000004CB6E711F4801F04BF01430020B4F12E
:1099E000FD0C88BFBCF5E06F3FF6AFAEB5EB030CE6
:1099F00004BFB6EB020C5FEA500C50F1000041EBE3
:109A0000045170BD0EF0004E4EEA113114EB5C04AF
:109A1000C2BFD4EB0C0541EA045170BD41F4801182
:109A20004FF0000E013C90E645EA060E8DE60CEA8A
:109A3000135594EA0C0F08BF95EA0C0F3FF43BAFA7
:109A400094EA0C0F0AD150EA01347FF434AF95EA5E
:109A50000C0F7FF425AF104619462CE795EA0C0F42
:109A600006D152EA03353FF4FDAE1046194622E70F
:109A700050EA410618BF52EA43067FF4C5AE50EAE9
:109A800041047FF40DAF52EA43057FF4EBAE12E7D9
:109A90004FF0FF3C06E000BF4FF0010C02E000BFBA
:109AA0004FF0010C4DF804CD4FEA410C7FEA6C5C9D
:109AB0004FEA430C18BF7FEA6C5C1BD001B050EA40
:109AC000410C0CBF52EA430C91EA030F02BF90EA2B
:109AD000020F0020704710F1000F91EA030F58BFEA
:109AE000994208BF90422CBFD8176FEAE37040F04C
:109AF000010070474FEA410C7FEA6C5C02D150EAEA
:109B0000013C07D14FEA430C7FEA6C5CD6D152EAA4
:109B1000033CD3D05DF8040B704700BF8446104669
:109B200062468C461946634600E000BF01B5FFF768
:109B3000B7FF002848BF10F1000F01BD4DF808ED38
:109B4000FFF7F4FF0CBF012000205DF808FB00BF09
:109B50004DF808EDFFF7EAFF34BF012000205DF863
:109B600008FB00BF4DF808EDFFF7E0FF94BF0120B0
:109B700000205DF808FB00BF4DF808EDFFF7CEFFB1
:109B800094BF012000205DF808FB00BF4DF808EDF0
:109B9000FFF7C4FF34BF012000205DF808FB00BFC1
:109BA0004FEA410C7FEA6C5C02D150EA013C0AD1D9
:109BB0004FEA430C7FEA6C5C02D152EA033C02D1CB
:109BC0004FF0000070474FF0010070474FEA41022C
:109BD00012F5001215D211D56FF47873B3EB6252FF
:109BE00012D94FEAC12343F0004343EA505311F026
:109BF000004F23FA02F018BF404270474FF00000B8
:109C0000704750EA013005D111F0004008BF6FF0F5
:109C1000004070474FF00000704700BF1FB51C4662
:109C2000094B1B680546D86852B1084B0091CDE935
:109C3000013207492B46224600F028F800F0B8FD13
:109C4000044B1A46F2E700BF5000002008CA00008B
:109C500015CA00008FB80000014B1868704700BF9C
:109C60005000002008B5074B044613B10021AFF3A4
:109C70000080054B1868836A03B19847204601F0BD
:109C800071FB00BF0000000044CA00000EB403B521
:109C9000014603AB054853F8042B0068019300F01C
:109CA0007FF802B05DF804EB03B07047500000206D
:109CB00070B50D4E0D4CA41BA4100025A54209D172
:109CC0000B4E0C4C01F050FBA41BA4100025A54228
:109CD00005D170BD56F8253098470135EEE756F8A6
:109CE000253098470135F2E72002002020020020AD
:109CF000200200203002002010B5431E0A44914289
:109D000000D110BD11F8014B03F8014FF7E788426D
:109D100010B501EB020307D8421E99420AD011F890
:109D2000014B02F8014FF8E78342F5D98118D21AA6
:109D3000D34200D110BD13F8014D01F8014DF7E7F2
:109D400002440346934200D1704703F8011BF9E730
:109D50009368013B002B10B4936007DA9469A34227
:109D600001DB0A2902D110BC00F062BC1368581C48
:109D700010601970084610BC7047F8B506460F46CB
:109D80001446D518AC4201D1002007E03A4614F839
:109D9000011B3046FFF7DCFF431CF3D1F8BD000088
:109DA0002DE9F04F9DB00C4617460393064618B1B7
:109DB00083690BB900F0F4FD7B4B9C4257D174686A
:109DC000A38918075DD52369002B5AD00023099376
:109DD00020238DF8293030238DF82A304FF0010BE5
:109DE000B846454615F8013B0BB1252B54D1B8EBCD
:109DF000070A0BD053463A4621463046FFF7BDFFCF
:109E0000013000F0C280099B5344099398F8003058
:109E1000002B00F0BA8000234FF0FF32CDE905237C
:109E2000049307938DF853301A93A846052218F827
:109E3000011B5E4800F0C4FE049B78BBD90644BFFA
:109E400020228DF853201A0744BF2B228DF853206F
:109E50002A782A2A2AD0079AA84600200A254146AD
:109E600011F8013B303B092B69D960B324E0504B1A
:109E70009C4201D1B468A3E74E4B9C4208BFF468F2
:109E80009EE72146304600F025FC00289ED04FF08A
:109E9000FF301DB0BDE8F08FA846A2E7434A801A04
:109EA0000BFA00F0184304904546BEE7039A111DD3
:109EB00012680391002A01DB079204E0524243F04A
:109EC00002030792049398F800302E2B0ED198F8D5
:109ED00001302A2B38D1039B1A1D1B680392002BDB
:109EE000B8BF4FF0FF3308F102080593324D98F8E0
:109EF00000100322284600F063FE40B14023401BBF
:109F000003FA00F0049B034308F10108049398F856
:109F100000102A488DF82810062208F1010700F0E9
:109F20004FFE002837D0264B1BBB039B073323F083
:109F3000070308330393099B4B44099350E705FB40
:109F40000232012088468AE7002308F101080593C0
:109F500019460A25404610F8012B303A092A03D940
:109F6000002BC3D00591C1E705FB012101238046E9
:109F7000F0E703AB00932246124B04A93046AFF33F
:109F80000080B0F1FF3F8146D5D1A3895B063FF544
:109F90007EAF09987DE703AB00932246094B04A9E5
:109FA000304600F087F8ECE79CCA000048CA000081
:109FB000BCCA00007CCA00004ECA000052CA0000A1
:109FC000000000007B9D00002DE9F04791461F46F0
:109FD0008A680B69DDF820809342B8BF1346C9F840
:109FE000003091F8432006460C4612B10133C9F8FF
:109FF00000302368990642BFD9F800300233C9F80F
:10A000000030256815F0060507D104F1190AE36848
:10A01000D9F800209B1AAB4228DC94F84330226820
:10A02000003318BF012392062DD404F143023946B0
:10A030003046C047013020D02368E568D9F80020B9
:10A0400003F00603042B08BFAD1AA36822690CBFF6
:10A0500025EAE57500259342C4BF9B1AED184FF021
:10A0600000091A344D451AD1002008E00123524658
:10A0700039463046C047013003D14FF0FF30BDE8CC
:10A08000F0870135C3E7E1185A1C302081F84300FE
:10A09000224494F8451082F843100233C5E70123A7
:10A0A000224639463046C0470130E6D009F1010961
:10A0B000D8E700002DE9F04301F1430C0C46097E7E
:10A0C00085B06E291746064698460C9A00F0B38074
:10A0D00022D8632936D00AD8002900F0B98058293F
:10A0E00000F0838004F1420584F8421032E06429D4
:10A0F00001D06929F6D120681368050603F104012F
:10A100002AD51B681160002B03DA2D225B4284F8EC
:10A1100043206F480A2239E0732900F09D8008D857
:10A120006F2920D07029DDD1236843F020032360FC
:10A1300003E0752917D07829D4D1782384F84530E5
:10A14000644855E01368191D1B68116004F142054D
:10A1500084F8423001238CE01B68116010F0400F3E
:10A1600018BF1BB2CFE713682568181D10602806BA
:10A1700001D51B6802E06806FBD51B8854486F298F
:10A1800014BF0A220822002184F843106568A560E4
:10A19000002DC0F29580216821F004012160002B80
:10A1A0003DD1002D40F08E806546082A0BD12368F2
:10A1B000DB0708D5236962689A42DEBF302305F8C1
:10A1C000013C05F1FF35ACEB05032361CDF80080C0
:10A1D0003B4603AA21463046FFF7F6FE01304DD13B
:10A1E0004FF0FF3005B0BDE8F083394884F84510E2
:10A1F000136821681D1D1B6815600A060BD5CA0768
:10A2000044BF41F0200121601BB9226822F02002E6
:10A2100022601022B7E74D0648BF9BB2EFE76546C4
:10A22000B3FBF2F102FB1133C35C05F8013D0B46B1
:10A230000029F5D1B9E7136825686169181D106018
:10A2400028061B6801D5196002E06A06FBD5198053
:10A25000002323616546B9E71368191D11601D6865
:10A2600062680021284600F0ABFC08B1401B60602A
:10A2700063682361002384F84330A7E723692A46F3
:10A2800039463046C0470130AAD023689B0713D413
:10A29000E068039B9842B8BF1846A3E701234A46EB
:10A2A00039463046C04701309AD00135E368039AF9
:10A2B0009B1AAB42F2DCEBE7002504F11909F5E744
:10A2C000002BACD1037884F8423004F142056CE7EE
:10A2D00059CA00006ACA000038B50D4B1C68A36B50
:10A2E00005467BB9182000F04DFC0A4A0A4BA063D2
:10A2F000C0E90023094B83600B23838101220023E3
:10A30000C0E90423A36B00221D615A6138BD00BF60
:10A31000500000200E33CDAB34126DE6ECDE0500AC
:10A3200038B5134B1C68A36B7BB9182000F02AFCCE
:10A33000104A114BA063C0E90023104B83600B232C
:10A34000838101220023C0E90423A16B0C480A6920
:10A350004B690C4C504304FB0300A2FB0423034451
:10A36000541C43F10005C1E9044525F0004038BD07
:10A37000500000200E33CDAB34126DE6ECDE05004C
:10A380002DF451582D7F954C0CB430B5174B0C1E45
:10A390009DB01D6808DA8B232B604FF0FF301DB095
:10A3A000BDE8304002B070474FF40273ADF814308E
:10A3B00014BF04F1FF332346049307934FF6FF7352
:10A3C00002900690ADF81630209A21AB02A92846DB
:10A3D000019300F06DFD431CBCBF8B232B60002C50
:10A3E000DDD0029B00221A70D9E700BF5000002088
:10A3F0000EB400B59CB01DAB029006906FF000410A
:10A40000094807910491094953F8042B0591006804
:10A41000019302A900F04CFD029B00221A701CB0AF
:10A420005DF804EB03B07047500000200802FFFF06
:10A4300010B503461A785C1C3AB9013B11F8012BA0
:10A4400003F8012F002AF9D110BD2346F2E7C9B263
:10A45000034610F8012B1AB18A42F9D11846704709
:10A46000002918BF0023F9E710F8012B11F8013B70
:10A47000012A28BF9A42F7D0D01A7047034613F832
:10A48000012B002AFBD1181A0138704710B56AB1A8
:10A490000139841810F8013B11F8012F934203D1C0
:10A4A000A04201D0002BF5D1981A10BD1046FCE750
:10A4B00070B50139044602B970BD234611F8015F39
:10A4C00003F8015B561E2DB91444A342F4D003F8DF
:10A4D000015BFAE71C463246EDE7F0B503787BB145
:10A4E000044623782046661C7BB14A1E631E12F880
:10A4F000015F4DB113F8017FAF423446F7D0F0E76A
:10A500000B78002B18BF0020F0BD1846FCE72DE9A2
:10A51000F0478046894692461E460F463D460898BB
:10A5200015F8014B00F0C6FA2044437813F00803F5
:10A5300032D12D2C32D17C78BD1C0122002E5DD071
:10A54000102E09D1302C07D12B7803F0DF03582BC4
:10A550004FD16C7810260235002A14BF4FF000410D
:10A560006FF000410027B1FBF6FC384606FB1C1ECD
:10A57000A4F13003092B17D81C46A64223DD7B1C0F
:10A5800007D084451CD301D1A64519DB00FB06404A
:10A59000012715F8014BEBE72F46BFE72B2C04BF33
:10A5A000BD1C7C781A46C9E7A4F14103192B01D8D8
:10A5B000373CE2E7A4F16103192B04D8573CDCE7F0
:10A5C0004FF0FF37E5E77B1C08D12223C8F80030A5
:10A5D0000846BAF1000F07D1BDE8F08702B140424A
:10A5E000BAF1000FF8D00FB105F1FF39CAF80090A9
:10A5F000F2E73024002EAFD10826ADE7302CA3D0EF
:10A600000A26A9E7084B37B51C68084D236A002BBA
:10A6100008BF2B46009313460A4601462046FFF723
:10A6200076FF03B030BD00BF50000020B400002012
:10A63000F8B50E461446054618B183690BB900F00B
:10A64000AFF9214B9C422AD16C68A369A360A3890E
:10A650001A072ED5236963B323692068C01A63697A
:10A66000F6B28342374604DC2146284600F02EF934
:10A6700028BBA368013BA36023685A1C22601E709C
:10A6800063690130834204D0A389DB0719D50A2E00
:10A6900017D12146284600F019F990B10FE00B4B75
:10A6A0009C4201D1AC68D0E7094B9C4208BFEC68E2
:10A6B000CBE72146284600F00DF80028CCD04FF01B
:10A6C000FF373846F8BD00BF9CCA0000BCCA000076
:10A6D0007CCA0000324B70B51D6806460C4625B199
:10A6E000AB6913B9284600F05BF92E4B9C420FD1A1
:10A6F0006C68B4F90C309AB215072CD4D00611D47A
:10A700000922326043F04003A3814FF0FF303EE066
:10A71000254B9C4201D1AC68EBE7244B9C4208BF1F
:10A72000EC68E6E7510712D5616B41B104F14403CF
:10A73000994202D0304600F093FA00236363A38964
:10A7400023F02403A3810023636023692360A3898A
:10A7500043F00803A38123694BB9A38903F4207351
:10A76000B3F5007F03D02146304600F0CBF9A28933
:10A7700012F001030CD00023A36063695B42A36164
:10A78000236953B9B4F90C3013F08000BAD170BD0D
:10A79000920758BF6369A360F2E70020F7E700BFA4
:10A7A000500000209CCA0000BCCA00007CCA000007
:10A7B00008B5062000F0AAFC012000F0D3FD00003F
:10A7C0008A892DE9F041054610070C4658D44B689C
:10A7D000002B05DC0B6C002B02DC0020BDE8F081B7
:10A7E000E66A002EF9D0002312F480522F68216A05
:10A7F0002B6032D0606DA3895A0705D56368C01AF3
:10A80000636B0BB1236CC01A00230246E66A216A0F
:10A810002846B047431CA38906D129681D2948D87A
:10A82000294ACA40D60744D500226260D904226969
:10A83000226004D5421C01D12B6803B96065616BAD
:10A840002F600029C9D004F14403994202D0284660
:10A8500000F006FA00206063C0E701232846B047F5
:10A86000411CC8D12B68002BC5D01D2B01D0162B45
:10A8700001D12F60B1E7A38943F04003A381ADE785
:10A880000F69002FA9D093070E6808BF4B690F60AE
:10A8900018BF0023A6EB07088B60B8F1000F9CDD02
:10A8A00043463A46216AA66A2846B047002806DC95
:10A8B000A38943F04003A3814FF0FF308EE70744A4
:10A8C000A8EB0008E9E700BF0100402038B50B699C
:10A8D00005460C46DBB118B183690BB900F060F88E
:10A8E0000C4B9C4209D16C68B4F90C307BB1214609
:10A8F0002846BDE83840FFF763BF074B9C4201D1B3
:10A90000AC68F1E7054B9C4208BFEC68ECE700201F
:10A9100038BD00BF9CCA0000BCCA00007CCA000051
:10A92000002310B50446C0E900338360818143668B
:10A93000C281C0E904338361194608225C30FFF705
:10A94000FFF9054B6362054BA362054BE362054BC0
:10A950002462236310BD00BF45B1000067B1000051
:10A960009FB10000C3B10000014900F085B800BFED
:10A97000CDA8000070B54A1E682555430E4605F166
:10A98000740100F0BBF9044640B10021C0E9001693
:10A990000C30A06005F16802FFF7D2F9204670BDC7
:10A9A000836910B5044633BBC0E912330365124B0B
:10A9B000124A1B688262984204BF0123836100F03F
:10A9C0001FF86060204600F01BF8A060204600F0F1
:10A9D00017F80022E06004216068FFF7A1FF012260
:10A9E0000921A068FFF79CFF02221221E068FFF70F
:10A9F00097FF0123A36110BD44CA000069A90000AC
:10AA0000F8B51B4B1E68B369074613B93046FFF70C
:10AA1000C7FF4836D6E90134013B03D5336833B16B
:10AA20003668F7E7B4F90C506DB16834F4E70421E7
:10AA30003846FFF79FFF30600028F1D10C233B60C0
:10AA400004462046F8BD0B4B6566C4E90055A56079
:10AA5000C4E90335C4E905550822294604F15C0020
:10AA6000FFF76EF9C4E90D55C4E91255E9E700BFD7
:10AA700044CA00000100FFFF2DE9F84380468946E3
:10AA800000F14804002614B93046BDE8F883D4E943
:10AA90000175013F01D52468F5E7AB89012B07D982
:10AAA000B5F90E30013303D029464046C847064366
:10AAB0006835EEE7D0F8EC00704770B50E46B1F996
:10AAC0000E10002996B014461D4607DA00232B60AD
:10AAD000B3891A0610D44FF480630EE06A4600F082
:10AAE000A3FB0028F2DB019A02F47042A2F50053A6
:10AAF0005A425A412A60EEE740230020236016B0F4
:10AB000070BD00008B8973B59D0706460C4607D5BE
:10AB100004F14703236023610123636102B070BD28
:10AB200001AB6A46FFF7C9FF00990546304600F0C1
:10AB3000E5F848B9B4F90C309A05EFD423F00303D3
:10AB400043F00203A381E3E70D4BB362A3892060C6
:10AB500043F08003A381009B6361019B20615BB193
:10AB6000B4F90E10304600F071FB28B1A38923F030
:10AB7000030343F00103A381A3891D43A581CDE70E
:10AB800069A90000024B0146186800F0B7B800BF81
:10AB90005000002082B001B901A942B14BB1137835
:10ABA0000B601278101C18BF012002B070471046CD
:10ABB000FBE76FF00100F8E7000000000000000074
:10ABC00001F0FF01102A2BDB10F0070F08D010F85E
:10ABD000013B013A8B422DD010F0070F42B3F6D162
:10ABE000F0B441EA012141EA014122F007047FF07B
:10ABF00000070023F0E80256083C85EA010586EAD2
:10AC0000010685FA47F5A3FA87F586FA47F6A5FA0D
:10AC100087F68EB9EED1F0BC01F0FF0102F0070219
:10AC200032B110F8013B013A83EA010313B1F8D1C4
:10AC30000020704701387047002D06BF35460338A5
:10AC4000073815F0010F07D1013015F4807F02BFDE
:10AC5000013015F4C03F0130F0BC0138704700BF2F
:10AC600038B50546002945D051F8043C0C1F002B8F
:10AC7000B8BFE41800F00CFB1F4A1368104633B944
:10AC8000636014602846BDE8384000F002BBA34270
:10AC90000CD921686218934204BF1A685B6863602C
:10ACA00004BF521822600460ECE713465A680AB1E8
:10ACB000A242FAD919685818A0420BD12068014461
:10ACC000581882421960DDD1106852685A600144F8
:10ACD0001960D7E702D90C232B60D3E7206821182D
:10ACE0008A4204BF11685268626004BF091821607B
:10ACF0005C60C7E738BD00BF607A012070B5CD1C2D
:10AD000025F0030508350C2D38BF0C25002D06460F
:10AD100001DBA94203D90C233360002070BD00F091
:10AD2000B7FA214A1468214691B9204C23681BB90F
:10AD3000304600F0B3F920602946304600F0AEF905
:10AD4000431C24D10C233360304600F0A2FAE4E720
:10AD50000B685B1B18D40B2B0FD90B60CD50CC1894
:10AD6000304600F096FA04F10B00231D20F0070096
:10AD7000C31AD3D05A42E250D0E78C424B6816BF78
:10AD8000636013600C46EBE70C464968CCE7C41CD3
:10AD900024F00304A04205D0211A304600F07EF9C9
:10ADA0000130CFD02560DBE7607A0120647A012092
:10ADB000F8B5074614460E4621B91146BDE8F840DD
:10ADC000FFF79CBF22B9FFF74BFF25462846F8BD89
:10ADD00000F060FAA0420FD221463846FFF78EFFFE
:10ADE00005460028F2D031462246FEF785FF31465F
:10ADF0003846FFF735FFE9E73546E7E72DE9F04745
:10AE00008E689E4282460C469046994637D88A897B
:10AE100012F4906F31D0256809696F1A65690223B1
:10AE200005EB450595FBF3F509F101033B449D4214
:10AE300038BF1D46530530D52946FFF75FFF06464C
:10AE400050B90C23CAF80030A38943F04003A38112
:10AE50004FF0FF30BDE8F0873A462169FEF74CFF1E
:10AE6000A38923F4906343F08003A3812661656185
:10AE70003E44ED1B2660A5604E464E4500D94E4629
:10AE8000324641462068FEF742FFA3689B1BA36041
:10AE900023681E4426600020DCE72A46FFF788FF6F
:10AEA00006460028E2D121695046FFF7D9FEC8E7DF
:10AEB0002DE9F04F9DB0804603938B891D060C460B
:10AEC00016460FD50B696BB94021FFF717FF2060BD
:10AED000206128B90C23C8F800304FF0FF30C7E0DC
:10AEE000402363610023099320238DF82930302308
:10AEF0008DF82A304FF0010B37463D4615F8013BDF
:10AF00000BB1252B3ED1B7EB060A0BD05346324688
:10AF100021464046FFF772FF013000F0A480099BF4
:10AF2000534409933B78002B00F09D8000234FF0A1
:10AF3000FF32CDE90523049307938DF853301A931C
:10AF40002F46052217F8011B4F48FFF739FE049BD7
:10AF5000D0B9D90644BF20228DF853201A0744BF28
:10AF60002B228DF853202A782A2A15D0079A2F46AB
:10AF700000200A25394611F8013B303B092B4DD9F9
:10AF8000B8B10FE02F46B8E73F4A801A0BFA00F03D
:10AF9000184304903D46D3E7039A111D12680391AC
:10AFA000002A01DB079204E0524243F002030792B9
:10AFB00004933B782E2B0CD17B782A2B33D1039B27
:10AFC0001A1D1B680392002BB8BF4FF0FF330237E6
:10AFD00005932E4D397803222846FFF7F1FD38B14D
:10AFE0004023401B03FA00F0049B03430137049302
:10AFF000397827488DF8281006227E1CFFF7E0FDDF
:10B00000002838D0234B13BB039B073323F00703DF
:10B0100008330393099B4B4409936DE705FB023208
:10B0200001200F46A6E700230137059319460A259C
:10B03000384610F8012B303A092A03D9002BC8D022
:10B040000591C6E705FB012101230746F0E703ABA5
:10B0500000932246104B04A94046AFF30080B0F1A4
:10B06000FF3F8146D6D1A3895B063FF536AF0998ED
:10B070001DB0BDE8F08F03AB00932246064B04A938
:10B080004046FFF717F8EAE748CA00004ECA00003A
:10B0900052CA000000000000FDAD000038B5064CAB
:10B0A000002305460846236000F046F9431C02D100
:10B0B000236803B12B6038BDF48D01201F2938B5FA
:10B0C00004460D4604D9162303604FF0FF3038BD07
:10B0D000426C12B152F821304BB9204600F030F8E2
:10B0E0002A4601462046BDE8384000F017B8012B3B
:10B0F0000AD0591C03D1162303600120E7E700247E
:10B1000042F82540284698470020E0E7024B0146D8
:10B110001868FFF7D3BF00BF5000002038B5074CB8
:10B120000023054608461146236000F0EDF8431C55
:10B1300002D1236803B12B6038BD00BFF48D01201C
:10B1400000F0D2B810B50C46B1F90E1000F0AAF814
:10B150000028ABBF636DA3891B1823F48053ACBFD9
:10B160006365A38110BD2DE9F0411F468B89DB0586
:10B1700005460C46164605D502230022B1F90E10ED
:10B1800000F074F8A389B4F90E1023F48053A3815E
:10B1900032463B462846BDE8F04100F023B810B5E2
:10B1A0000C46B1F90E1000F061F8431CA38915BFDD
:10B1B000606523F4805343F48053A38118BFA381B7
:10B1C00010BDB1F90E1000F01FB849B1FF2A85BFBC
:10B1D0008A2303600A704FF0FF3098BF0120704748
:10B1E0000846704738B5074C054608461146002208
:10B1F00022601A4600F0AEF8431C02D1236803B166
:10B200002B6038BDF48D012038B5064C002305466F
:10B210000846236000F058F8431C02D1236803B1AC
:10B220002B6038BDF48D012038B5074C002305464E
:10B2300008461146236000F04FF8431C02D12368F2
:10B2400003B12B6038BD00BFF48D012038B5064C2A
:10B25000002305460846236000F04EF8431C02D147
:10B26000236803B12B6038BDF48D012038B5074C3D
:10B27000054608461146002222601A4600F04CF8A6
:10B28000431C02D1236803B12B6038BDF48D01202B
:10B290007047704751F8043C181F002BBCBF0B5877
:10B2A000C018704738B5074C0546084611460022BD
:10B2B00022601A4600F038F8431C02D1236803B11B
:10B2C0002B6038BDF48D0120024B58221A604FF0DC
:10B2D000FF307047F48D0120024B58221A604FF066
:10B2E000FF307047F48D0120024B58221A604FF056
:10B2F000FF307047F48D0120024B58221A60002065
:10B30000704700BFF48D0120024B58221A604FF0A5
:10B31000FF307047F48D0120024B58221A604FF025
:10B32000FF307047F48D0120024B58221A604FF015
:10B33000FF307047F48D0120044A05491368002B43
:10B3400008BF0B461844106018467047687A012001
:10B35000F88D0120024B58221A604FF0FF307047E1
:10B36000F48D0120FEE700BFF8B500BFF8BC08BCB3
:10B370009E467047F8B500BFF8BC08BC9E467047B3
:10B38000646174610000000004B400001D05000049
:10B390000DB400000D06000015B40000E90B00001C
:10B3A0001CB40000F90C000021B4000043080000A8
:10B3B0002CB400007706000031B40000350F000007
:10B3C0003DB400004F05000047B40000010B000031
:10B3D00055B40000CF09000062B400000B08000063
:10B3E00072616E646F6D00616C6C006C61737400EF
:10B3F00066616C7365007472756500252E31357356
:10B400002E2E2E006D616B654C697374006164644F
:10B410004C6173740064656C657465006A6F696E75
:10B4200000636F707946726F6D546F0066696E6469
:10B43000006A6F696E537472696E677300756E6926
:10B44000636F6465417400756E69636F64655374FE
:10B4500072696E67006E65774279746541727261D8
:10B460007900667265654D656D6F72790000000048
:10B47000D5B40000CD130000DAB40000E7130000DB
:10B4800015B40000EB130000E0B40000D11300007D
:10B49000EAB40000EF130000F3B40000F31300005F
:10B4A000FDB40000F713000008B50000FB13000016
:10B4B00014B50000D51300001DB50000DF13000017
:10B4C00027B50000D913000032B50000E3130000D7
:10B4D00066696C65006F70656E00636C6F73650004
:10B4E000656E644F6646696C6500726561644C699F
:10B4F0006E65007265616442797465730061707095
:10B50000656E644C696E6500617070656E64427949
:10B510007465730066696C6553697A65007374615C
:10B5200072744C697374006E657874496E4C6973FB
:10B53000740073797374656D496E666F0000000066
:10B54000201600003016000044160000B816000057
:10B55000EA1600001A1700004C1700006E170000D2
:10B56000AA170000E217000032180000721800004D
:10B57000DA18000018190000381900006C190000D2
:10B58000AC190000CE190000F8190000221A0000C2
:10B59000621A0000DA1A0000A21B0000141C00004E
:10B5A0005E1C0000C01C0000DC1C0000FA1C000037
:10B5B000941D0000D01D0000401E00006E1E000003
:10B5C000961E0000CE1E0000321F0000961F0000D5
:10B5D000DA1F00001E2000008E200000FE20000068
:10B5E000482100008C210000C2210000062200003A
:10B5F0004C22000092220000E42200003A230000C6
:10B6000078230000EC2300002024000066240000C2
:10B61000AC240000F22400002C250000722500005C
:10B62000B825000014270000F81900006C1900006C
:10B630002C26000020160000602600008626000050
:10B64000BA260000E02600002016000020160000A8
:10B6500020160000201600008A270000CA270000DC
:10B660000E2800006228000088280000D62800006C
:10B67000FC2800002C2900002016000020160000E5
:10B680004A2900007C290000AE290000E2290000C0
:10B69000062A00003A2A0000882A0000AA2A000090
:10B6A000CC2A0000FE2A0000302B0000542B0000A2
:10B6B000782B0000AA2B0000CE2B000020160000E3
:10B6C00020160000201600002016000020160000A2
:10B6D000002C0000262C00004C2C0000722C0000D6
:10B6E000982C0000CC2C0000002D0000342D000010
:10B6F000682D00008E2D0000B42D0000E82D000004
:10B700002016000020160000201600002016000061
:10B710002016000020160000201600002016000051
:10B720002016000020160000201600002016000041
:10B7300020160000201600000E2E00003E2E0000F5
:10B740005B2564206974656D206C6973745D0028E5
:10B7500025642062797465732900286F626A6563C5
:10B760007420747970653A202564290053746163EC
:10B770006B20756E646572666C6F7700626F6F6CBC
:10B7800065616E006E756D62657200737472696ECC
:10B7900067006C697374006279746520617272610C
:10B7A00079000000070000000300000005B8000059
:10B7B000592F00000DB800000530000016B8000039
:10B7C000A33000001FB800005D2F000028B8000063
:10B7D000A730000030B800009530000000000000E5
:10B7E000010000000200000003000000040000004F
:10B7F0000A0000001D0000006D6963726F3A626903
:10B800007420763200686173546F6E6500706C61ED
:10B8100079546F6E6500686173536572766F00735B
:10B820006574536572766F00646163496E69740074
:10B83000646163577269746500474320746F6F6B6E
:10B840002025642075736563733B206672656520EF
:10B85000256420776F726473003C496E7465676578
:10B86000723E003C4C6973743E003C4F626A6563F3
:10B87000743E003C4279746541727261793E000DFC
:10B880000A564D2050616E69633A2025730D0A00F7
:10B890006D69736300000000CDB80000DD3D00005D
:10B8A000D6B80000613D0000DAB80000AD3C0000F1
:10B8B000E2B800004F3C0000ECB80000E13B0000A3
:10B8C000F8B80000E33A00006E756C6C00686578AB
:10B8D000546F496E740073696E006A736F6E4765CA
:10B8E00074006A736F6E436F756E74006A736F6E67
:10B8F00056616C75654174006A736F6E4B65794172
:10B900007400000060B900003D3E000068B900000E
:10B91000413E000072B90000533E00007BB90000B8
:10B92000593E000086B900005F3E000092B9000059
:10B93000653E0000A7B900006B3E0000BCB90000E6
:10B94000713E0000C8B90000773E0000D8B9000081
:10B95000473E0000E4B900004D3E00006E657400F3
:10B9600068617357694669007374617274576946F8
:10B97000690073746F705769466900776966695327
:10B980007461747573006D794950416464726573B4
:10B99000730068747470536572766572476574528B
:10B9A00065717565737400726573706F6E64546F42
:10B9B000487474705265717565737400687474703E
:10B9C000436F6E6E65637400687474704973436F7F
:10B9D0006E6E656374656400687474705265717529
:10B9E0006573740068747470526573706F6E7365FC
:10B9F0000000000004000000030000000A00000036
:10BA00000700000006000000000000000008080811
:10BA100000080A4A4000000A5FEA5FEA0ED92ED306
:10BA20006E19324489330C924C924D080800000084
:10BA300004880808040804848488000A448A4000B2
:10BA4000048EC480000000048800000EC0000000C6
:10BA500000080001224488100C9252524C048C843D
:10BA6000848E1C824C901E1EC244924C06CA525FA9
:10BA7000E21FF01EC13E02448ED12E1FE244881008
:10BA80000ED12ED12E0ED12EC48800080008000041
:10BA9000048004880244880482000EC00EC008049A
:10BAA0008244880ED126C0040ED135B36C0C925E50
:10BAB000D2521C925C925C0ED010100E1C9252520C
:10BAC0005C1ED01C901E1ED01C90100ED013712E28
:10BAD00012525ED2521C8808081C1FE242524C12BD
:10BAE00054981492101010101E113B75B131113979
:10BAF00035B3710C9252524C1C925C90100C9252C5
:10BB00004C861C925C92510ED00C825C1FE48484A3
:10BB100084125252524C1131312A44113135BB71C9
:10BB200012524C9252112A4484841EC488101E0E54
:10BB3000C808080E10080482410EC242424E048A10
:10BB4000400000000000001F0804800000000ED22A
:10BB5000524F10101C925C000ED0100E02424ED2BA
:10BB60004E0C925C900E06C81C88080ED24EC24C39
:10BB700010101C92520800080808024002424C10A3
:10BB8000149814920808080806001B75B131001CAF
:10BB9000925252000C92524C001C925C90000ED2B9
:10BBA0004EC2000ED010100006C8049808080EC837
:10BBB00007001252524F0011312A4400113135BB97
:10BBC00000124C8C9200112A4498001EC4881E0654
:10BBD000C48C8486080808080818080C8818000017
:10BBE0000C83600000000000010000000200000063
:10BBF0000300000004000000050000000600000033
:10BC00000700000008000000090000000A00000012
:10BC10000B0000000C0000000D0000000E000000F2
:10BC20000F000000100000001200000014000000CF
:10BC300016000000180000001A0000001C000000A0
:10BC40001E0000002000000023000000260000006D
:10BC5000290000002C0000002F000000320000002E
:10BC6000360000003A0000003E00000042000000E4
:10BC7000460000004B00000050000000550000008E
:10BC80005A00000061000000680000006F00000022
:10BC9000760000007D000000840000008B000000A2
:10BCA0009200000099000000A0000000A700000022
:10BCB000AE000000B5000000BC000000C3000000A2
:10BCC000CA000000D1000000D8000000DF00000022
:10BCD000E6000000ED000000F4000000FB000000A2
:10BCE000FF0000000000000002000000040000004F
:10BCF00001000000030000005CBD0000913E000058
:10BD000067BD00000143000071BD00004D3F000011
:10BD10007EBD00006D41000085BD0000B9410000FE
:10BD20008EBD0000094200009ABD0000FD400000E9
:10BD3000ABBD0000A13F0000B8BD00008540000081
:10BD40001500000016000000170000001800000099
:10BD500019000000646973706C6179006C69676830
:10BD6000744C6576656C006D62446973706C6179C2
:10BD7000006D62446973706C61794F6666006D6234
:10BD8000506C6F74006D62556E706C6F74006D62F4
:10BD9000447261775368617065006D6253686170C9
:10BDA00065466F724C6574746572006E656F50699C
:10BDB00078656C53656E64006E656F506978656C6C
:10BDC00053657450696E004E6F7420656E6F7567B1
:10BDD0006820726F6F6D206576656E206166746590
:10BDE0007220636F6D70616374696F6E00436F6D75
:10BDF00070616374656420466C61736820636F646E
:10BE0000652073746F72650A2564206279746573A6
:10BE1000207573656420282564252529206F6620F8
:10BE2000256400426164207265636F726420666FEE
:10BE3000756E6420647572696E6720696E697469D5
:10BE4000616C697A6174696F6E00256420256420D5
:10BE500025642028256420776F7264732900256487
:10BE6000207265636F7264732C20256420776F7273
:10BE700064732C206D617849442025642C20636F05
:10BE80006D70616374696F6E206379636C65732094
:10BE9000256400526573746F726564202564207395
:10BEA00063726970747300537461727465640072B4
:10BEB0006164696F0000000048BF0000F14B0000A2
:10BEC00055BF0000654E000065BF0000F94D000041
:10BED00073BF0000C54F00007EBF0000194C00007A
:10BEE0008EBF0000A94C0000A2BF00008D4C0000D6
:10BEF000B1BF0000A1510000BDBF00001D510000F6
:10BF0000C6BF0000C1500000D1BF000011500000AA
:10BF1000DCBF000049500000E5BF00007950000080
:10BF2000EEBF0000294C0000FDBF0000094C0000DE
:10BF300006C00000394C00006E6F6E65006F7468BB
:10BF4000657200706169720064697361626C655248
:10BF50006164696F006D65737361676552656365E0
:10BF600069766564007061636B65745265636569C9
:10BF70007665007061636B657453656E640072650D
:10BF8000636569766564496E74656765720072659C
:10BF90006365697665644D6573736167655479702F
:10BFA00065007265636569766564537472696E676E
:10BFB0000073656E64496E74656765720073656EC3
:10BFC00064506169720073656E64537472696E6760
:10BFD000007365744368616E6E656C0073657447C9
:10BFE000726F757000736574506F77657200736956
:10BFF000676E616C537472656E6774680064657611
:10C000006963654944006C6173744D65737361675E
:10C0100065494400556E6B6E6F776E207072696D66
:10C020006974697665205B25733A25735D000000AD
:10C0300000000000963007772C610EEEBA51099986
:10C0400019C46D078FF46A7035A563E9A395649EE2
:10C050003288DB0EA4B8DC791EE9D5E088D9D29706
:10C060002B4CB609BD7CB17E072DB8E7911DBF9062
:10C070006410B71DF220B06A4871B9F3DE41BE8486
:10C080007DD4DA1AEBE4DD6D51B5D4F4C785D383E2
:10C0900056986C13C0A86B647AF962FDECC9658A86
:10C0A0004F5C0114D96C0663633D0FFAF50D088DE2
:10C0B000C8206E3B5E10694CE44160D5727167A286
:10C0C000D1E4033C47D4044BFD850DD26BB50AA5E2
:10C0D000FAA8B5356C98B242D6C9BBDB40F9BCAC06
:10C0E000E36CD832755CDF45CF0DD6DC593DD1AB62
:10C0F000AC30D9263A00DE518051D7C81661D0BF86
:10C10000B5F4B42123C4B3569995BACF0FA5BDB8E1
:10C110009EB802280888055FB2D90CC624E90BB185
:10C12000877C6F2F114C6858AB1D61C13D2D66B6E1
:10C130009041DC760671DB01BC20D2982A10D5EF45
:10C140008985B1711FB5B606A5E4BF9F33D4B8E8A1
:10C15000A2C9077834F9000F8EA8099618980EE145
:10C16000BB0D6A7F2D3D6D08976C6491015C63E6A1
:10C17000F4516B6B62616C1CD83065854E0062F2C5
:10C18000ED95066C7BA5011BC1F4088257C40FF521
:10C19000C6D9B06550E9B712EAB8BE8B7C88B9FC45
:10C1A000DF1DDD62492DDA15F37CD38C654CD4FBA1
:10C1B0005861B24DCE51B53A7400BCA3E230BBD445
:10C1C00041A5DF4AD795D83D6DC4D1A4FBF4D6D3A1
:10C1D0006AE96943FCD96E34468867ADD0B860DA45
:10C1E000732D0444E51D03335F4C0AAAC97C0DDDA1
:10C1F0003C710550AA41022710100BBE86200CC9C5
:10C2000025B56857B3856F2009D466B99FE461CE20
:10C210000EF9DE5E98C9D9292298D0B0B4A8D7C744
:10C22000173DB359810DB42E3B5CBDB7AD6CBAC0A0
:10C230002083B8EDB6B3BF9A0CE2B6039AD2B174BC
:10C240003947D5EAAF77D29D1526DB048316DC7318
:10C25000120B63E3843B64943E6A6D0DA85A6A7ABC
:10C260000BCF0EE49DFF099327AE000AB19E077D18
:10C2700044930FF0D2A3088768F2011EFEC206693C
:10C280005D5762F7CB67658071366C19E7066B6E98
:10C29000761BD4FEE02BD3895A7ADA10CC4ADD67BC
:10C2A0006FDFB9F9F9EFBE8E43BEB717D58EB06018
:10C2B000E8A3D6D67E93D1A1C4C2D83852F2DF4FBC
:10C2C000F167BBD16757BCA6DD06B53F4B36B24818
:10C2D000DA2B0DD84C1B0AAFF64A0336607A0441BC
:10C2E000C3EF60DF55DF67A8EF8E6E3179BE694618
:10C2F0008CB361CB1A8366BCA0D26F2536E268523C
:10C3000095770CCC03470BBBB91602222F26055597
:10C31000BE3BBAC5280BBDB2925AB42B046AB35CBB
:10C32000A7FFD7C231CFD0B58B9ED92C1DAEDE5B17
:10C33000B0C2649B26F263EC9CA36A750A936D02FB
:10C34000A906099C3F360EEB856707721357000557
:10C35000824ABF95147AB8E2AE2BB17B381BB60C7B
:10C360009B8ED2920DBED5E5B7EFDC7C21DFDB0BD7
:10C37000D4D2D38642E2D4F1F8B3DD686E83DA1FFB
:10C38000CD16BE815B26B9F6E177B06F7747B71857
:10C39000E65A0888706A0FFFCA3B06665C0B0111FB
:10C3A000FF9E658F69AE62F8D3FF6B6145CF6C1657
:10C3B00078E20AA0EED20DD75483044EC2B30339FB
:10C3C000612667A7F71660D04D476949DB776E3E57
:10C3D0004A6AD1AEDC5AD6D9660BDF40F03BD8377B
:10C3E00053AEBCA9C59EBBDE7FCFB247E9FFB530D7
:10C3F0001CF2BDBD8AC2BACA3093B353A6A3B424FB
:10C400000536D0BA9306D7CD2957DE54BF67D92356
:10C410002E7A66B3B84A61C4021B685D942B6F2AFA
:10C4200037BE0BB4A18E0CC31BDF055A8DEF022D56
:10C43000416C6C207461736B732073746F707065E2
:10C4400064007631303700202573202573004D6558
:10C450006D6F727920636C6561726564004E6F2048
:10C4600066726565207461736B20656E74726965B0
:10C4700073000000CCC40000E9660000D9C40000CD
:10C4800065610000E5C40000B9660000EBC400006F
:10C49000C9660000F1C40000D9660000F7C40000BE
:10C4A0009561000001C500003167000009C500006A
:10C4B0008564000012C500001D6200001AC500005E
:10C4C000B563000073656E736F72730061636365BB
:10C4D0006C65726174696F6E0074656D7065726110
:10C4E000747572650074696C74580074696C745961
:10C4F0000074696C745A00746F7563685265616486
:10C50000006932635265616400693263577269740D
:10C51000650072656164444854006D6963726F70B0
:10C52000686F6E65000000009CC50000B1670000E8
:10C53000AAC50000B5670000B3C50000C1670000D0
:10C54000BDC50000C5670000C6C50000C967000082
:10C55000CBC50000CD670000D0C50000D16700004A
:10C56000DCC50000D5670000E3C50000D967000006
:10C57000ECC50000DD670000F1C50000E1670000C8
:10C58000FCC50000E567000006C60000B9670000B2
:10C5900010C60000BD67000074667400656E6162BD
:10C5A0006C65446973706C61790067657457696480
:10C5B00074680067657448656967687400736574BA
:10C5C000506978656C006C696E6500726563740013
:10C5D000726F756E6465645265637400636972633B
:10C5E0006C6500747269616E676C6500746578745F
:10C5F00000746674546F756368656400746674547F
:10C600006F7563685800746674546F756368590079
:10C61000746674546F756368507265737375726570
:10C62000007661727300000048C60000496C00008B
:10C6300052C60000296C00005BC60000056C0000BB
:10C6400067C60000976B0000766172457869737465
:10C6500073007661724E616D656400736574566136
:10C66000724E616D6564007661724E616D65466FF4
:10C6700072496E6465780057656C636F6D652074F0
:10C680006F204D6963726F426C6F636B7321007032
:10C690005F73706920213D204E554C4C002F686F10
:10C6A0006D652F6769742F2E706C6174666F726D83
:10C6B000696F2F7061636B616765732F6672616D5F
:10C6C00065776F726B2D61726475696E6F6E6F72D4
:10C6D0006469636E7266352F6C6962726172696536
:10C6E000732F5350492F5350492E6370700053508D
:10C6F00049436C6173733A3A535049436C617373A5
:10C70000284E52465F5350495F547970652A2C2059
:10C7100075696E74385F742C2075696E74385F7437
:10C720002C2075696E74385F7429000000000000C9
:10C7300000000000496E0000016E0000376E00002E
:10C740003D6E0000436E0000356E000002000000E8
:10C7500003000000040000001F0000001C00000097
:10C760000E000000250000000B0000000A00000081
:10C77000090000001E000000170000000C0000006F
:10C7800011000000010000000D0000002200000068
:10C79000FFFFFFFFFFFFFFFF1A0000002000000067
:10C7A00015000000160000000F0000001800000037
:10C7B000130000002400000000000000140000002E
:10C7C0000500000010000000080000001900000033
:10C7D000060000002800000000000000000000002B
:10C7E0000F750000F57B0000857500009175000055
:10C7F0008B7500000D75000005750000997500002F
:10C80000297500000175000000C0014000100240C1
:10C810000020024000000000000000000000304343
:10C8200000000000000030C373717274000000004B
:10C83000FB21F93FFB2109407CD91240FB21194023
:10C840007A6A1F407CD92240BBFD2540FB2129404C
:10C850003A462C407A6A2F405C4731407CD93240BE
:10C860009C6B3440BBFD3540DB8F3740FB213940AA
:10C870001BB43A403A463C405AD83D407A6A3F4061
:10C880004C7E40405C4741406C1042407CD9424065
:10C890008CA243409C6B4440AC344540BBFD4540BA
:10C8A000CBC64640DB8F4740EB584840FB21494010
:10C8B00083F9A200444E6E00FC291500D1572700D1
:10C8C000DD34F50062DBC0003C99950041904300E7
:10C8D0006351FE00BBDEAB00B761C5003A6E2400B9
:10C8E000D24D42004906E00009EA2E001C92D10018
:10C8F000EB1DFE0029B11C00E83EA700F5358200C3
:10C9000044BB2E009CE98400B4267000417E5F0089
:10C91000D6913900538339009CF439008B5F840031
:10C9200028F9BD00F81F3B00DEFF97000F980500B7
:10C93000112FEF000A5A8B006D1F6D00CF7E36005D
:10C9400009CB2700464FB7009E663F002DEA5F00E7
:10C95000BA277500E5EBC7003D7BF100F73907000A
:10C9600092528A00FB6BEA001FB15F00085D8D00E8
:10C97000300356007BFC4600F0AB6B0020BCCF00C0
:10C9800036F49A00E3A91D005E619100081BE600E1
:10C9900085996500A0145F008D40680080D8FF0075
:10C9A00027734D0006063100CA561500C9A873004A
:10C9B0007BE260006B8CC00000000040FB21F93F6F
:10C9C000000000002D44743E000000809846F83CB2
:10C9D0000000006051CC783B00000080831BF039E0
:10C9E0000000004020257A38000000802282E336D3
:10C9F000000000001DF36935020000000300000084
:10CA000004000000060000002C2066756E63746947
:10CA10006F6E3A2000617373657274696F6E2022C5
:10CA2000257322206661696C65643A2066696C65CD
:10CA300020222573222C206C696E652025642573C5
:10CA400025730A0054000020232D302B2000686C31
:10CA50004C00656667454647003031323334353621
:10CA6000373839414243444546003031323334355A
:10CA70003637383961626364656600000000000083
:10CA800000000000000000000000000000000000A6
:10CA90000000000000000000000000000000000096
:10CAA0000000000000000000000000000000000086
:10CAB0000000000000000000000000000000000076
:10CAC0000000000000000000000000000000000066
:10CAD0000000000000000000000000004300504F74
:10CAE00053495800002020202020202020202828E2
:10CAF000282828202020202020202020202020201E
:10CB0000202020202088101010101010101010105D
:10CB1000101010101004040404040404040404108D
:10CB2000101010101010414141414141010101011B
:10CB300001010101010101010101010101010101E5
:10CB400010101010101042424242424202020202F1
:10CB500002020202020202020202020202020202B5
:10CB60001010101020000000000000000000000065
:10CB700000000000000000000000000000000000B5
:10CB800000000000000000000000000000000000A5
:10CB90000000000000000000000000000000000095
:10CBA0000000000000000000000000000000000085
:10CBB0000000000000000000000000000000000075
:10CBC0000000000000000000000000000000000065
:10CBD0000000000000000000000000000000000055
:0CCBE00000000000000000000000000049
:08CBEC005438FF7F0100000036
:10CBF400FFFFFFFFD007000001000000E803DC0591
:10CC0400DC05DC05DC050000FFFFFFFFFFFFFFFF85
:10CC14001800000019FCFFFFFFFFFFFFFF000000EA
:10CC24000090D003FFFFFFFFFFFFFFFFFFFFFFFFA9
:10CC34000A000000010000000800000001000000DC
:10CC440054000020000000009CCA0000BCCA000080
:10CC54007CCA00000000000000000000000000008A
:10CC640000000000000000000000000000000000C0
:10CC740000000000000000000000000000000000B0
:10CC840000000000000000000000000000000000A0
:10CC94000000000000000000000000000000000090
:10CCA400000000004300000000000000000000003D
:10CCB4000000000000000000000000000000000070
:10CCC400000000004300000000000000000000001D
:10CCD4000000000000000000000000000000000050
:10CCE40000000000430000000000000000000000FD
:10CCF4000000000000000000000000000000000030
:10CD040000000000430000000000000000000000DC
:10CD1400000000000000000000000000000000000F
:10CD240000000000430000000000000000000000BC
:10CD340000000000000000000000000000000000EF
:10CD4400000000004300000000000000000000009C
:10CD540000000000000000000000000000000000CF
:10CD6400000000004300000000000000000000007C
:10CD740000000000000000000000000000000000AF
:10CD840000000000CBB1000095AB000000000000E3
:10CD9400E4CA000002B400008FB800008FB800009D
:10CDA4008FB800008FB800008FB800008FB8000063
:10CDB4008FB800008FB800008FB80000FFFFFFFF9E
:10CDC400FFFFFFFFFFFFFFFFFFFF000001004153D4
:10CDD400434949000000000000000000000000007A
:10CDE40000000000000000000000000000004153AB
:10CDF400434949000000000000000000000000005A
:10CE0400000000000000000000000000000000001E
:10CE140025040000CD6D0000297200009977000000
:04CE24000104000005
:04000003000072E5A2
:00000001FF
